:100000000C94BB010C9427320C9454320C94E301F1
:100010000C94E3010C94E3010C94E3010C94E301D0
:100020000C94E3010C94E3010C94E3010C94CE06D0
:100030000C94E3010C94E3010C94E3010C94E301B0
:100040000C9433310C94E3010C9444060C94800618
:100050000C94E3010C94E3010C94E3010C94E30190
:100060000C94E3010C94E301084AD73B3BCE016EAC
:1000700084BCBFFDC12F3D6C74319ABD56833DDAFF
:100080003D00C77F11BED9E4BB4C3E916BAAAABE0E
:10009000000000803F05A84CCDB2D44EB93836A937
:1000A000020C50B9918688083CA6AAAA2ABE000074
:1000B00000803F0664EC1B3C04BC163E3BE5B93CAB
:1000C000C93C37C29E5A3D660498083EEA69AAAA0E
:1000D0003E000000803F2020BF0020BF00BF007C0A
:1000E0002020202020202020202020202020202010
:1000F00020202000C8202020202020202020202078
:1001000020C900C8202020202020202020202020BE
:10011000C97C00D820202020202020202020202042
:10012000D97C00C820202020202020202020202032
:10013000C97C00C820202020202020202020202032
:10014000C97C00207265766F00206172737369004C
:100150006D696E6F706F7364206C6962726570692F
:100160006C6F74002020202020BABBBCBDBE7C2058
:1001700020202020CACBCCCDCE7C00626F6F74696A
:100180006E672075703AEDF2F2F2F2F2F2F2F300DD
:1001900062617474657279207761726E696E67202E
:1001A0000074787069642076616C756573006261B3
:1001B000726F2074656D700074656D706469737022
:1001C00020006163746976652000706173736976DD
:1001D000650075617674616C6B2000736574757071
:1001E0002073637265656E7C7C7C0043686172205D
:1001F000446F6E650A00526561647920666F7220F3
:10020000466F6E740A0055706461746520436861BE
:10021000725365740000407A10F35A00A0724E18B1
:10022000090010A5D4E80000E87648170000E40BA8
:1002300054020000CA9A3B000000E1F5050000806E
:10024000969800000040420F000000A086010000C8
:1002500000102700000000E8030000000064000018
:100260000000000A00000000000100000000002C57
:1002700076D888DC674F0823DFC1DFAE59E1B1B71C
:1002800096E5E3E453C63AE651997696E8E6C284E9
:1002900026EB898C9B62ED407C6FFCEFBC9C9F4001
:1002A000F2BAA56FA5F490055A2AF75C936B6CF926
:1002B000676DC11BFCE0E40D47FEF520E6B500D0FC
:1002C000ED902E0300943577050080841E08000011
:1002D000204E0A000000C80C333333330F986E12DF
:1002E000831141EF8D2114893BE65516CFFEE6DBE5
:1002F00018D1844B381BF77C1D901DA4BBE424202F
:100300003284725E228100C9F124ECA1E53D276EA2
:10031000616E00696E660000000000240027002A5C
:100320000000000000250028002B00000000002332
:100330000026002900040404040404040402020248
:100340000202020303030303030102040810204016
:10035000800102040810200102040810200000009F
:100360000700020100000304060000000000000076
:1003700000004F04150811241FBECFEFD8E0DEBFE8
:10038000CDBF14E0A0E0B1E0E0E4FFE602C00590DC
:100390000D92A030B107D9F716E0A0E0B4E001C09B
:1003A0001D92A33BB107E1F713E0C6E7D3E004C019
:1003B0002297FE010E949A37C237D107C9F70E94DF
:1003C00063330C949E370C940000FA01AA2728305E
:1003D00051F1203181F1E8946F936E7F6E5F7F4F12
:1003E0008F4F9F4FAF4FB1E03ED0B4E03CD0670F8E
:1003F000781F891F9A1FA11D680F791F8A1F911DE1
:10040000A11D6A0F711D811D911DA11D20D009F430
:1004100068943F912AE0269F11243019305D319372
:10042000DEF6CF010895462F4770405D4193B3E05B
:100430000FD0C9F7F6CF462F4F70405D4A3318F002
:10044000495D31FD4052419302D0A9F7EACFB4E0B3
:10045000A6959795879577956795BA95C9F700976B
:100460006105710508959B01AC010A2E069457950C
:10047000479537952795BA95C9F7620F731F841F63
:10048000951FA01D0895283008F027E03327DA01D2
:10049000990F311D87FD916000966105710539F452
:1004A00032602E5F3D9330E32A95E1F708959F3F38
:1004B00030F080387105610509F03C5F3C5F3D9389
:1004C000913008F08068911DDF93CF931F930F93B5
:1004D000FF92EF92192F987F9695E92F9695969512
:1004E000E90FFF27E159FD4F99273327EE24FF2419
:1004F000A701E70105900894079428F4360FE71E3A
:10050000F81E491F511D660F771F881F991F0694FB
:10051000A1F70590079428F4E70EF81E491F561F0F
:10052000C11D770F881F991F661F0694A1F70590BC
:10053000079428F4F80E491F561FC71FD11D880FB6
:10054000991F661F771F0694A1F70590079420F462
:10055000490F561FC71FD81F990F661F771F881F87
:100560000694A9F784911095177041F0D695C79518
:1005700057954795F794E7941A95C1F7E5E1F2E0AE
:1005800068941590159135916591959105907FE24C
:100590007395E118F10A430B560BC90BD009C0F74C
:1005A000E10CF11E431F561FC91FD01D7EF470338E
:1005B00011F48A95E6CFE894015030F0080F0AF460
:1005C0000027021708F4202F2395022F7A3328F0F2
:1005D00079E37D932A95E9F710C07D932A9589F6F2
:1005E000069497956795379517951794E118F10A32
:1005F000430B560BC90BD00998F023957E91739548
:100600007A3308F070E37C932013B8F77E91706121
:100610007D9330F0839571E37D9370E32A95E1F744
:100620001124EF90FF900F911F91CF91DF919927A7
:1006300087FD90950895CF93DF93BC01823091059B
:1006400010F462E070E0A091B106B091B206ED0145
:1006500040E050E0E0E0F0E021C088819981861719
:10066000970769F48A819B81309719F0938382837D
:1006700004C09093B2068093B106FE0134C068179F
:10068000790738F44115510519F08417950708F4D6
:10069000AC01FE018A819B819C01E9012097E9F66A
:1006A00041155105A9F1CA01861B970B049708F45F
:1006B000BA01E0E0F0E02AC08D919C911197841777
:1006C0009507F9F46417750781F412968D919C9142
:1006D0001397309719F09383828304C09093B206E6
:1006E0008093B106FD0132964CC0CA01861B970B60
:1006F000FD01E80FF91F6193719302978D939C930D
:1007000040C0FD01828193819C01D9011097A1F61F
:100710008091AF069091B006892B41F48091A002A0
:100720009091A1029093B0068093AF064091A202EF
:100730005091A3024115510541F44DB75EB7809128
:100740009E0290919F02481B590B2091AF06309159
:10075000B006CA01821B930B8617970780F0AB0186
:100760004E5F5F4F8417950750F0420F531F509311
:10077000B0064093AF06F9016193719302C0E0E0C7
:10078000F0E0CF01DF91CF910895CF93DF930097F1
:1007900009F450C0EC0122971B821A82A091B10685
:1007A000B091B206109709F140E050E0AC17BD07D8
:1007B00008F1BB83AA83FE0121913191E20FF31F5F
:1007C000AE17BF0779F48D919C911197280F391FAF
:1007D0002E5F3F4F3983288312968D919C911397FA
:1007E0009B838A834115510571F4D093B206C0935F
:1007F000B10620C012968D919C911397AD01009780
:1008000011F0DC01D3CFFA01D383C283219131915E
:10081000E20FF31FCE17DF0769F488819981280F53
:10082000391F2E5F3F4FFA01318320838A819B81DC
:1008300093838283DF91CF910895FC0105906150ED
:1008400070400110D8F7809590958E0F9F1F0895E6
:10085000FC016150704001900110D8F7809590958F
:100860008E0F9F1F08956EBD0DB407FEFDCF8EB590
:1008700008958DE061E00E9481328BE061E00E948A
:1008800081328CE060E00E9481328AE061E00E9467
:1008900081321CBC80E58CBD8DB58EB5089580E09D
:1008A00094E00E9439040895FC011382128288EEBC
:1008B00093E0A0E0B0E084839583A683B78385EBC3
:1008C00092E0918380830895FC018089803419F43B
:1008D00021E030E002C020E030E0C9010895FC01D1
:1008E000818990E00895FC01648745876687478782
:1008F000089580E090E0089580E090E0089580E021
:1009000090E008950895EF92FF921F93CF93DF93A5
:10091000162F7A0186E060E00E94C03280E094E009
:1009200060E00E94330480E094E060E00E943304C1
:1009300080E094E069E00E94330480E094E0612F5D
:100940000E943304C0E0D0E0F701EC0FFD1F1081DE
:1009500080E094E06AE00E94330480E094E06C2F31
:100960000E94330480E094E06BE00E94330480E056
:1009700094E0612F0E9433042196C633D10521F7FC
:1009800080E094E068E00E94330480E094E060EA54
:100990000E94330480E094E060EA0E94330485FD05
:1009A000F9CF80E094E060E00E94330480E094E0BE
:1009B0006CE00E94330486E061E00E94C032DF9167
:1009C000CF911F91FF90EF9008951F93CF93DF93E6
:1009D000EC01162F86E060E00E94C03280E094E0D7
:1009E00060E00E943304112319F0113059F404C05F
:1009F00080E094E0688904C068896C6180E094E0DC
:100A00000E94330486E061E00E94C032DF91CF9102
:100A10001F910895EF92FF920F931F938EE1489FCD
:100A200070011124E60EF11C86E060E00E94C032E5
:100A300000E014E0C80165E00E943304C8016F2D96
:100A40000E943304C80166E00E943304C8016E2D81
:100A50000E9433041F910F91FF90EF900895EF9241
:100A6000FF920F931F937C0100E014E0C80167E040
:100A70000E943304C8016FEF0E94330486E061E0F6
:100A80000E94C032F70187858F5F87871F910F9182
:100A9000FF90EF900895EF92FF920F931F93FC0148
:100AA000E7848EE1E89E700111248685E80EF11C32
:100AB00086E060E00E94C03200E014E0C80164E01B
:100AC0000E943304C80163E00E943304C80165E05A
:100AD0000E943304C8016F2D0E943304C80166E0F0
:100AE0000E943304C8016E2D0E9433041F910F91A0
:100AF000FF90EF9008951F93CF93DF93EC01162F93
:100B00006C3731F40E942F05CE010E944B050AC0BC
:100B100080E094E067E00E94330480E094E0612F7D
:100B20000E94330481E090E0DF91CF911F910895FE
:100B30000F931F9386E060E00E94C03200E014E053
:100B4000C80164E00E943304C80164E00E943304D9
:100B500086E061E00E94C0321F910F9108951F93BB
:100B6000CF93DF93EC01188A16E0198B8FE996E09A
:100B700060E973E00E949330813049F480E4888B0F
:100B800088E0898B86E060E00E94C03202C0188A4B
:100B9000198B86E060E00E94C032DF91CF911F91F7
:100BA00008950F931F93CF93DF93EC0186E061E0EC
:100BB0000E94813282E060E00E94813282E061E046
:100BC0000E94C032CE010E94AF0586E060E00E9424
:100BD000C03280E094E06CEE0E94330480E094E048
:100BE0006FEF0E943304182F80E094E060E00E94D1
:100BF00033046889626080E094E00E94330462E319
:100C000070E080E090E00E94893180E094E06CE642
:100C10000E9433041F7E80E094E0612F0E94330421
:100C20008889803419F00DE010E002C000E110E086
:100C3000109202041092010417C060910104709197
:100C40000204605F80E094E00E94330480E094E05E
:100C500069E00E943304809101049091020401969E
:100C60009093020480930104809101049091020406
:100C70008017910714F3CE0161E00E94E504DF9133
:100C8000CF911F910F9108951F920F920FB60F925F
:100C900011242F933F934F938F939F93EF93FF9341
:100CA0004091C60020918E0630918F062F5F3F4FF6
:100CB0008091920690919306282339238091900683
:100CC000909191062817390779F080918E069091BE
:100CD0008F06E0919406F0919506E80FF91F408386
:100CE00030938F0620938E06FF91EF919F918F9105
:100CF0004F913F912F910F900FBE0F901F9018951D
:100D00001F920F920FB60F9211242F933F938F9340
:100D10009F93EF93FF9320919806309199068091CD
:100D200096069091970628173907E9F08091980662
:100D300090919906E0919C06F0919D06E80FF91FAD
:100D400080818093C60080919806909199060196C3
:100D500020919A0630919B068223932390939906C3
:100D60008093980610C02091960630919706809146
:100D70009806909199062817390729F48091C100A7
:100D80008F7D8093C100FF91EF919F918F913F9153
:100D90002F910F900FBE0F901F9018951F920F92DA
:100DA0000FB60F9211248F939F938091C30490915B
:100DB000C404892B51F08091C5049091C60401961A
:100DC0009093C6048093C50409C08091C704909194
:100DD000C80401969093C8048093C7049F918F9193
:100DE0000F900FBE0F901F901895CF93DF93482F51
:100DF000EB0180912406833009F45DC0843028F42F
:100E00008130C1F0823058F50AC0853009F4D2C073
:100E1000853008F4A8C0863009F0F2C0E9C04C3330
:100E200009F0EEC081E080932406488384EB809330
:100E30002306E6C0842F90E0E0912306F0E0E82747
:100E4000F927ED53FD4F208120932306887F907072
:100E5000809741F582E080932406498329C0242F9E
:100E600030E0E0912306F0E0E227F327ED53FD4F59
:100E7000808180932306809122068F5F80932206D3
:100E8000823018F43B832A83BBC0922F88272A81A3
:100E90003B81820F931F9B838A830A978F3F910523
:100EA00021F018F010922406ABC083E08093240652
:100EB00010922206A5C0E42FF0E08091230690E076
:100EC000E827F927ED53FD4F808180932306609139
:100ED00022066F5F60932206623089F0633020F44F
:100EE000613009F08DC006C0633091F0643009F0C4
:100EF00087C022C0842F90E0A0E0B0E018C0242F6B
:100F000030E040E050E0542F432F322F222707C01B
:100F1000242F30E040E050E0A901332722278C81C4
:100F20009D81AE81BF81820F931FA41FB51F8C834B
:100F30009D83AE83BF8364C0242F30E040E050E047
:100F4000522F4427332722278C819D81AE81BF8178
:100F5000820F931FA41FB51F8C839D83AE83BF8315
:100F600060932406A5CF242F30E0E0912306F0E023
:100F7000E227F327ED53FD4F808180932306809174
:100F800022068F5F80932206813019F08230C1F5EE
:100F900003C03987288734C0922F88272885398550
:100FA000280F391F398728878A819B810A97F1F09A
:100FB00085E07CCFE42FF0E08091230690E0E827E5
:100FC000F927ED53FD4F808180932306209122065F
:100FD0002F5F2093220630E0FB01E20FF31F4187D1
:100FE0008A819B810A972817390750F086E05ECFE7
:100FF000C75FDE4F4883C950D14087E08093240605
:1010000080912406873069F410922406C75FDE4F72
:10101000909123068881C950D140981711F48A8194
:1010200001C080E0DF91CF9108958F92AF92CF926F
:10103000EF92FF920F931F9389E894E060E045ECF4
:1010400050E024EC30E000EC10E0B1ECEB2EF12CA1
:10105000CC24C394A8E9AA2EF0E28F2E0E94032A82
:1010600086EA94E00E9454041092B9041092BA04E3
:101070001092BB041092BC041092BD041092BE04E6
:101080001092BF041092C0041092C2041092C104C6
:101090001092B8041F910F91FF90EF90CF90AF90F6
:1010A0008F900895AF92BF92CF92DF92EF92FF920E
:1010B0000F931F93E0908A06F0908B0600918C06A8
:1010C00010918D068FE590E0A0E0B0E0E80EF91EEB
:1010D0000A1F1B1F0E947B316E157F058007910739
:1010E00008F44EC0A090EE04B090EF04C090F0045D
:1010F000D090F104C601B50120E030E040E85FE3A4
:101100000E940336181694F5E0904206F0904306CC
:1011100000914406109145060E947B3120918A0679
:1011200030918B0640918C0650918D06621B730B9B
:10113000840B950B0E94D9349B01AC01C601B5010B
:101140000E940E3620E030E04AE754E40E9440342A
:101150009B01AC01C801B7010E9473336093420642
:101160007093430680934406909345060E947B311A
:1011700060938A0670938B0680938C0690938D06FD
:101180001F910F91FF90EF90DF90CF90BF90AF90A5
:101190000895DF93CF9300D000D0CDB7DEB7FB0129
:1011A000E80FF91F628583859485258569838A8385
:1011B0009B832C83492F5C81782FCA010F900F905D
:1011C0000F900F90CF91DF910895AF92BF92DF9271
:1011D000EF92FF920F931F93CF93DF938C01809137
:1011E000250680FDE4C0F801F08089E894E06F2DC9
:1011F0000E94E42AE801C75FDE4FEF2DF0E0ED53D7
:10120000FD4F80818883F801F18089E894E06F2D9B
:101210000E94E42AEF2DF0E0888190E0E827F9278A
:10122000ED53FD4F80818883F801F28089E894E0D6
:101230006F2D0E94E42AEF2DF0E0888190E0E827EE
:10124000F927ED53FD4F80818883F801F38089E809
:1012500094E06F2D0E94E42AEF2DF0E0888190E069
:10126000E827F927ED53FD4F80818883F801F4804A
:1012700089E894E06F2D0E94E42AEF2DF0E0888148
:1012800090E0E827F927ED53FD4F80818883F8012E
:101290002481358146815781232F342F452F5527AF
:1012A000F22E89E894E0622F0E94E42AEF2DF0E00C
:1012B000888190E0E827F927ED53FD4F80818883EE
:1012C000F80124813581468157819A0144275527A9
:1012D000F22E89E894E0622F0E94E42AEF2DF0E0DC
:1012E000888190E0E827F927ED53FD4F80818883BE
:1012F000F8012481358146815781252F33274427E2
:101300005527F22E89E894E0622F0E94E42AEF2DFF
:10131000F0E0888190E0E827F927ED53FD4F8081C8
:10132000888389E894E060E00E94E42AE881F0E0A4
:10133000ED53FD4F8081888389E894E060E00E944E
:10134000E42AE881F0E0ED53FD4F80818883F801C5
:10135000828193810B9718F18AE0A82EB12CA00E00
:10136000B11E750112C0F701D1907F0189E894E0A8
:101370006D2D0E94E42AED2DF0E0888190E0E827B1
:10138000F927ED53FD4F808188832E2D2A1930E0F7
:10139000F801828193810A972817390720F3075FA4
:1013A0001E4F89E894E0F80160810E94E42ADF91F1
:1013B000CF911F910F91FF90EF90DF90BF90AF9072
:1013C0000895DF93CF93CDB7DEB7CA50D1400FB6A3
:1013D000F894DEBF0FBECDBF2CE329836A832AE0D9
:1013E00030E03C832B83FC0184819581A681B78109
:1013F0008D839E83AF83B887CE0101960E94E50856
:10140000C65FDE4F0FB6F894DEBF0FBECDBFCF91E3
:10141000DF9108958FE996E06AE773E00E949330C8
:10142000882331F586E696E6A6E6B0E480932706A3
:1014300090932806A0932906B0932A0680E090E0B6
:10144000A0E8BFE380932B0690932C06A0932D0673
:10145000B0932E0688EE93E09093300680932F068B
:1014600081E8809331068DE8809332068DEF25C0A8
:1014700082E598EBAEE0B0E48093270690932806CF
:10148000A0932906B0932A0685E89BEEA1E5B0E477
:1014900080932B0690932C06A0932D06B0932E06D6
:1014A00080EA94E19093300680932F068BEF80932F
:1014B000310686E6809332068AEF809333060895DC
:1014C000FF920F931F930FE916E0C8016CE773E0DA
:1014D0000E94933080936E06C8016EE773E00E940D
:1014E000933080936F06C80160E873E00E949330E8
:1014F00080934E06C8016EE873E00E94933080939B
:101500006606C8016AE873E00E949330809364061F
:10151000C80164E873E00E94933080937006C801AC
:1015200066E873E00E94933080937106C8016CE80E
:1015300073E00E94933080935606C80162E973E01D
:101540000E94933080937206C80164E973E00E94A0
:10155000933080935506C80164EF73E00E94933086
:10156000F82EC80165EF73E00E949330382F20E019
:101570002F0D311D3093740620937306C80166EF5A
:1015800073E00E949330F82EC80167EF73E00E9469
:101590009330382F20E02F0D311D309376062093A5
:1015A0007506C80168EF73E00E949330F82EC801F9
:1015B00069EF73E00E949330382F20E02F0D311D2A
:1015C0003093780620937706C8016BEF73E00E9492
:1015D000933080934D061F910F91FF900895BC01A9
:1015E0008FE996E00E94933008956091D80470913D
:1015F000D9048091DA049091DB0420E030E040E1EE
:1016000052E40E940E3620E030E044EB53E40E94A6
:1016100040340E9471360E94A8349B01255030400E
:1016200037FF03C09B01215E3F4FA6E3B6E0F901FF
:10163000ED53FC4F80818C932F5F3F4F2432310557
:1016400014F020E030E0119686E0A134B80779F775
:101650001C9208952F923F924F925F926F927F92C9
:101660008F929F92AF92BF92CF92DF92EF92FF92B2
:101670000F931F93DF93CF9300D000D000D0CDB74E
:10168000DEB7182F662E2091CE043091CF042A3574
:10169000310530F0C9018D549F4F89359105E8F42B
:1016A00037FF02C02D543F4FC90137FF03C090954B
:1016B00081959F4F8A3191053CF0F4E48F2E912C57
:1016C000E9ED2E2E312C1DC00A975CF17BE3872EAD
:1016D000912C62ED262E312C20C02B35310514F0D3
:1016E000235B3040C90137FF03C0909581959F4F20
:1016F0008A31910554F056E5852E912C4CED242E1F
:10170000312C37E0A32EB12C15C00A9754F02DE4EC
:10171000822E912C94ED292E312C88E0A82EB12C0C
:1017200009C005E0802E912CB8E32B2E312CA9E0C6
:10173000AA2EB12C6091D0047091D104882777FD36
:101740008095982F0E94DB3427EA32E94BE25CEB6C
:101750000E940E360E94E23620E030E040EA50E47B
:101760000E940E3620E030E040E951E40E940E363F
:101770000E94713620E030E044E352E40E9473336B
:101780000E94A834712EFEEBCF2EFFEFDF2E9B01BF
:10179000442737FD4095542F29833A834B835C833C
:1017A000E6EA4E2EE4E05E2E4AEF5FEF240E351E91
:1017B0006091CE047091CF04882777FD8095982F93
:1017C0000E94DB3425E33AEF4EE85CE30E940E36DC
:1017D0000E94E2367B018C01B601882777FD809557
:1017E000982F0E94DB349B01AC01C801B7010E9415
:1017F0000E367B018C0169817A818B819C810E94EC
:10180000DB349B01AC01C801B7010E9473330E9415
:10181000A8349B01CB0101978A35910508F071C06E
:1018200062E170E00E9448378B012F5F3F4FAEEEC0
:10183000BFEF6A9FC0016B9F900D7A9F900D11249E
:10184000820F931F62E070E00E9448376D837E83B1
:10185000E62CE01A4E2D4C5F86EA94E0672D0E943C
:101860000A0500D000D000D0EDB7FEB73196ADB775
:10187000BEB712965C924E92119720E031E033830E
:1018800022838D819E81880D991D958384830E947A
:10189000E2294DB75EB74A5F5F4F0FB6F8945EBF5F
:1018A0000FBE4DBF8D819E818A159B0554F104307A
:1018B00011053CF593E0E90EC201672D4E2D0E9403
:1018C0000A0500D000D000D0EDB7FEB73196ADB715
:1018D000BEB712965C924E92119720E031E03383AE
:1018E00022834D815E81420D531D558344830E94A6
:1018F000E2298DB79EB706960FB6F8949EBF0FBE2D
:101900008DBFACE0B0E0CA0EDB1E7394BEE4CB1614
:10191000D10409F04DCF26960FB6F894DEBF0FBE66
:10192000CDBFCF91DF911F910F91FF90EF90DF908E
:10193000CF90BF90AF909F908F907F906F905F906F
:101940004F903F902F900895823010F422E002C013
:10195000282F220F30E08DB79EB708970FB6F89466
:101960009EBF0FBE8DBFEDB7FEB7319686EA94E0FD
:10197000ADB7BEB712969C938E93119783E091E01A
:101980009383828322573F4F358324832F5F3F4FBA
:10199000378326830E94E2298DB79EB708960FB63B
:1019A000F8949EBF0FBE8DBF0895CF93DF93AC0117
:1019B000E091E004F091E104209134063091350685
:1019C000C9018C599F4F8E179F071CF4EA0121977C
:1019D00009C024563040E217F30714F0EA0102C0B0
:1019E000EA012196842F90E0C817D90729F08FE9E2
:1019F00096E04C2F0E949A30CE01DF91CF9108954E
:101A00000F931F930FE916E0C80163EF73E041E005
:101A10000E949A30C80164EF73E043E10E949A305B
:101A2000C80165EF73E046E00E949A30C80166EF96
:101A300073E040E10E949A30C80167EF73E047E22B
:101A40000E949A30C80168EF73E048E80E949A301B
:101A5000C80169EF73E043E10E949A301F910F9132
:101A60000895CF92DF92EF92FF920F931F937C0124
:101A7000D62EC72E06EA14E0C8016E2D4D2D0E9409
:101A80007304C8010E944B0500D000D0EDB7FEB72B
:101A90001283018383E391E0948383830E94D1299D
:101AA000EDB7FEB71283018383E291E094838383D1
:101AB0000E94D129EDB7FEB71283018383E191E043
:101AC000948383830E94D129EDB7FEB712830183EB
:101AD00083E091E0948383830E94D129EDB7FEB720
:101AE0001283018384EF90E0948383830E94D12941
:101AF0000F900F900F900F90C8010E942F05C70103
:101B000001966D2D7C2D0E942A0B1F910F91FF9045
:101B1000EF90DF90CF900895AF92BF92CF92DF9277
:101B2000EF92FF920F931F93B82EA62E0E947B3147
:101B300028EE33E040E050E00E945B3779018A01F3
:101B4000A6EACA2EA4E0DA2EC6016B2D4A2D0E9409
:101B50007304C6010E944B05A090FE04B090FF04E0
:101B60008DB79EB744970FB6F8949EBF0FBE8DBF3A
:101B7000EDB7FEB73196ADB7BEB71296DC92CE92F6
:101B8000119788E091E09383828383EB90E09583C3
:101B90008483C7016CE370E00E944837CB016CE39B
:101BA00070E00E944837978386832AE330E03187CC
:101BB0002087C7016CE370E00E94483793878287D3
:101BC00085E690E095878487C5016CE370E00E940C
:101BD0003437CB016CE370E00E94483797878687E3
:101BE000318B208BC5016CE370E00E943437938BFE
:101BF000828B0E94E2298DB79EB744960FB6F89467
:101C00009EBF0FBE8DBFC6010E942F051F910F9171
:101C1000FF90EF90DF90CF90BF90AF900895EF923C
:101C2000FF920F931F93282F462FB6EAEB2EB4E0B6
:101C3000FB2EC701622F0E947304C7010E944B054F
:101C40008DB79EB70A970FB6F8949EBF0FBE8DBF93
:101C50000DB71EB70F5F1F4FEDB7FEB7F282E182DF
:101C600080E291E0F8019383828360910005709196
:101C70000105809102059091030520912B0630917A
:101C80002C0640912D0650912E060E940E36F8012A
:101C9000648375838683978380EB90E09187808748
:101CA0000E94E2298DB79EB70A960FB6F8949EBFA0
:101CB0000FBE8DBFC7010E942F051F910F91FF908E
:101CC000EF9008958F929F92AF92BF92CF92DF9242
:101CD000EF92FF920F931F93E82EF62E06EA14E080
:101CE000C8016E2D4F2D0E947304C8010E944B0540
:101CF0008DB79EB70C970FB6F8949EBF0FBE8DBFE1
:101D0000EDB7FEB73196ADB7BEB712961C930E93E2
:101D1000119728E2822E21E0922E938282829DEEFC
:101D2000A92EB12CB582A4828091090590910A0553
:101D3000A0910B05B0910C0586839783A087B1878E
:101D400083EFC82ED12CD386C2860E94E2298DB79C
:101D50009EB70C960FB6F8949EBF0FBE8DBFC801FC
:101D60000E942F05F394C8016E2D4F2D0E9473041D
:101D7000C8010E944B05ADB7BEB71C970FB6F894CB
:101D8000BEBF0FBEADBFEDB7FEB7319612961C9326
:101D90000E93119793828282B582A48280910D0561
:101DA00090910E05A0910F05B09110058683978341
:101DB000A087B187D386C2860E94E2298DB79EB7DD
:101DC0000C960FB6F8949EBF0FBE8DBFC8010E943F
:101DD0002F05F394C8016E2D4F2D0E947304C80186
:101DE0000E944B05ADB7BEB71C970FB6F894BEBFA7
:101DF0000FBEADBFEDB7FEB7319612961C930E9392
:101E0000119793828282B582A4828091110590916C
:101E10001205A0911305B091140586839783A087BE
:101E2000B187D386C2860E94E2298DB79EB70C96F1
:101E30000FB6F8949EBF0FBE8DBFC8010E942F053C
:101E40001F910F91FF90EF90DF90CF90BF90AF90D8
:101E50009F908F9008950F931F93282F462F06EA87
:101E600014E0C801622F0E947304C8010E944B0550
:101E70008DB79EB70A970FB6F8949EBF0FBE8DBF61
:101E8000EDB7FEB73196ADB7BEB712961C930E9361
:101E9000119782E391E09383828389EB90E09583AD
:101EA00084838091FC049091FD049783868382E86B
:101EB00090E0918780870E94E2298DB79EB70A96AD
:101EC0000FB6F8949EBF0FBE8DBFC8010E942F05AC
:101ED0001F910F910895EF92FF920F931F93282F58
:101EE000462F36EAE32E34E0F32EC701622F0E941C
:101EF0007304C7010E944B058DB79EB70C970FB6B0
:101F0000F8949EBF0FBE8DBF0DB71EB70F5F1F4F5A
:101F1000EDB7FEB7F282E1828AE391E0F8019383A4
:101F2000828384EE90E0958384836091FA047091BB
:101F3000FB04882777FD8095982F0E94DB342AE0E8
:101F400037ED43E25CE30E940E36F8016683778347
:101F5000808791878FE890E0938782870E94E229AB
:101F60008DB79EB70C960FB6F8949EBF0FBE8DBF6F
:101F7000C7010E942F051F910F91FF90EF900895C8
:101F80000F931F93282F462F06EA14E0C801622FF3
:101F90000E947304C8010E944B058DB79EB70C9731
:101FA0000FB6F8949EBF0FBE8DBFEDB7FEB731964A
:101FB000ADB7BEB712961C930E9311978AE391E0CA
:101FC0009383828382EE90E0958384838091F604EC
:101FD0009091F704A091F804B091F9048683978357
:101FE000A087B1878EE890E0938782870E94E229DC
:101FF0008DB79EB70C960FB6F8949EBF0FBE8DBFDF
:10200000C8010E942F051F910F9108950F931F93F0
:10201000282F462F86EA94E0622F0E94730486EAF6
:1020200094E00E944B058091DD04882319F424E498
:1020300031E057C0813019F428E431E052C08230D9
:1020400019F42CE431E04DC0833019F420E531E07F
:1020500048C0843019F424E531E043C0853019F4D8
:1020600028E531E03EC0863019F42CE531E039C076
:10207000873019F420E631E034C0883019F424E6C2
:1020800031E02FC0893019F428E631E02AC08A30C7
:1020900019F42CE631E025C08B3019F420E731E04B
:1020A00020C08C3019F424E731E01BC08D3019F4C6
:1020B00028E731E016C08E3019F42CE731E011C06A
:1020C0008F3019F420E831E00CC0803119F424E895
:1020D00031E007C0813119F028E831E002C029E879
:1020E00031E08DB79EB708970FB6F8949EBF0FBE2C
:1020F0008DBFEDB7FEB7319606EA14E0ADB7BEB7B7
:1021000012961C930E9311978DE891E0938382832E
:1021100080EE90E095838483378326830E94E229B2
:102120008DB79EB708960FB6F8949EBF0FBE8DBFB1
:10213000C8010E942F051F910F9108950F931F93BF
:10214000282F462F06EA14E0C801622F0E9473046C
:10215000C8010E944B058DB79EB70A970FB6F89439
:102160009EBF0FBE8DBFEDB7FEB73196ADB7BEB700
:1021700012961C930E93119782E991E093838283C8
:1021800087E890E0958384838091DE049091DF045A
:102190009783868385E290E0918780870E94E22979
:1021A0008DB79EB70A960FB6F8949EBF0FBE8DBF2F
:1021B000C8010E942F051F910F9108950F931F933F
:1021C000282F462F06EA14E0C801622F0E947304EC
:1021D000C8010E944B058DB79EB70A970FB6F894B9
:1021E0009EBF0FBE8DBFEDB7FEB73196ADB7BEB780
:1021F00012961C930E9311978CE991E0938382833E
:102200008091D0049091D1049583848380EB90E0F9
:102210009783868381EB90E0918780870E94E229F3
:102220008DB79EB70A960FB6F8949EBF0FBE8DBFAE
:10223000C8010E942F051F910F9108950F931F93BE
:10224000282F462F06EA14E0C801622F0E9473046B
:10225000C8010E944B058DB79EB70A970FB6F89438
:102260009EBF0FBE8DBFEDB7FEB73196ADB7BEB7FF
:1022700012961C930E9311978CE991E093838283BD
:102280008091CE049091CF049583848380EB90E07D
:102290009783868382EB90E0918780870E94E22972
:1022A0008DB79EB70A960FB6F8949EBF0FBE8DBF2E
:1022B000C8010E942F051F910F9108950F931F933E
:1022C000282F462F06EA14E0C801622F0E947304EB
:1022D000C8010E944B058DB79EB70A970FB6F894B8
:1022E0009EBF0FBE8DBFEDB7FEB73196ADB7BEB77F
:1022F00012961C930E93119784EA91E09383828344
:1023000081EE90E0958384838091AC029091AD0240
:102310009783868385E290E0918780870E94E229F7
:102320008DB79EB70A960FB6F8949EBF0FBE8DBFAD
:10233000C8010E942F051F910F9108950F931F93BD
:10234000282F462F06EA14E0C801622F0E9473046A
:10235000C8010E944B058DB79EB70C970FB6F89435
:102360009EBF0FBE8DBFEDB7FEB73196ADB7BEB7FE
:1023700012961C930E9311978CEA91E093838283BB
:1023800086EB91E09583848380ED90E0978386834C
:1023900086E396E09187808781ED90E0938782873E
:1023A0000E94E2298DB79EB70C960FB6F8949EBF97
:1023B0000FBE8DBFC8010E942F051F910F91089578
:1023C0000F931F93282F462F06EA14E0C801622FAF
:1023D0000E947304C8010E944B058DB79EB70A97EF
:1023E0000FB6F8949EBF0FBE8DBFEDB7FEB7319606
:1023F000ADB7BEB712961C930E93119784EC91E083
:10240000938382838091D8049091D904A091DA04B7
:10241000B091DB0484839583A683B78380EB90E03F
:10242000918780870E94E2298DB79EB70A960FB6E2
:10243000F8949EBF0FBE8DBFC8010E942F051F914B
:102440000F9108950F931F93282F462F06EA14E04B
:10245000C801622F0E947304C8010E944B058DB70A
:102460009EB70C970FB6F8949EBF0FBE8DBFEDB709
:10247000FEB73196ADB7BEB712961C930E93119767
:102480008CEC91E09383828386E190E09583848352
:102490008091F2049091F304A091F404B091F504BA
:1024A00086839783A087B18788E890E093878287A7
:1024B0000E94E2298DB79EB70C960FB6F8949EBF86
:1024C0000FBE8DBFC8010E942F051F910F91089567
:1024D000CF92DF92EF92FF920F931F93CF93DF93F0
:1024E000282F462FC6EAD4E0CE01622F0E94730443
:1024F000CE010E944B056091420670914306809187
:1025000044069091450620912B0630912C0640916F
:102510002D0650912E060E940E366B017C0120E0A4
:1025200030E04AE754E40E9403361816D4F58DB71C
:102530009EB70C970FB6F8949EBF0FBE8DBF0DB718
:102540001EB70F5F1F4FADB7BEB71296DC93CE9389
:1025500011978AE391E0F801938382838EEF90E0F4
:102560009583848360912F0670913006882777FDCC
:102570008095982F0E94DB349B01AC01C701B60106
:102580000E944034D80116966D937D938D939C9351
:102590001997809133061A968C931A971B961C9262
:1025A00021C08DB79EB70C970FB6F8949EBF0FBE93
:1025B0008DBFEDB7FEB73196ADB7BEB71296DC93BF
:1025C000CE93119786ED91E0938382838EEF90E016
:1025D00095838483C682D782E086F1868091320615
:1025E000828713860E94E229EDB7FEB73C960FB6AC
:1025F000F894FEBF0FBEEDBF86EA94E00E942F055F
:10260000DF91CF911F910F91FF90EF90DF90CF90CE
:102610000895EF92FF920F931F93282F462F56EAAB
:10262000E52E54E0F52EC701622F0E947304C70106
:102630000E944B058DB79EB70C970FB6F8949EBFBE
:102640000FBE8DBF0DB71EB70F5F1F4FEDB7FEB7A3
:10265000F282E1828CEC91E0F8019383828389EE2F
:1026600090E0958384836091EE047091EF048091F3
:10267000F0049091F10420912706309128064091B2
:10268000290650912A060E940E36F8016683778348
:102690008087918780913106828713860E94E22984
:1026A0008DB79EB70C960FB6F8949EBF0FBE8DBF28
:1026B000C7010E942F051F910F91FF90EF90089581
:1026C000EF92FF920F931F93282F462F66EAE62E74
:1026D00064E0F62EC701622F0E947304C7010E94B6
:1026E0004B058DB79EB70C970FB6F8949EBF0FBEE3
:1026F0008DBF0DB71EB70F5F1F4FEDB7FEB7F2824C
:10270000E18286ED91E0F8019383828386EE90E08A
:10271000958384836091EA047091EB048091EC04CA
:102720009091ED0420912B0630912C0640912D06BE
:1027300050912E060E940E36F801668377838087BB
:10274000918780913206828713860E94E2298DB795
:102750009EB70C960FB6F8949EBF0FBE8DBFC701F3
:102760000E942F051F910F91FF90EF900895EF9217
:10277000FF920F931F93282F462F76EAE72E74E0DF
:10278000F72EC701622F0E947304C7010E944B05F8
:102790008DB79EB70C970FB6F8949EBF0FBE8DBF36
:1027A0000DB71EB70F5F1F4FEDB7FEB7F282E18284
:1027B00086ED91E0F8019383828387EE90E0958324
:1027C00084836091040570910505882777FD8095C5
:1027D000982F0E94DB3420912B0630912C064091DB
:1027E0002D0650912E060E940E36F80166837783DF
:1027F0008087918780913206828713860E94E22922
:102800008DB79EB70C960FB6F8949EBF0FBE8DBFC6
:10281000C7010E942F051F910F91FF90EF9008951F
:102820000F931F93282F462F06EA14E0C801622F4A
:102830000E947304C8010E944B05809146060E94C5
:10284000A40CC8010E942F051F910F910895EF92CB
:10285000FF920F931F93282F462FE6EAEE2EE4E017
:10286000FE2EC701622F0E947304C7010E944B0510
:102870008DB79EB70C970FB6F8949EBF0FBE8DBF55
:102880000DB71EB70F5F1F4FEDB7FEB7F282E182A3
:1028900086ED91E0F801938382838FE190E0958348
:1028A0008483609147067091480680914906909113
:1028B0004A060E94DB3420912B0630912C06409171
:1028C0002D0650912E060E940E36F80166837783FE
:1028D0008087918780913206828713860E94E22941
:1028E0008DB79EB70C960FB6F8949EBF0FBE8DBFE6
:1028F000C7010E942F051F910F91FF90EF9008953F
:102900000F931F93282F462F06EA14E0C801622F69
:102910000E947304C8010E944B058DB79EB7409773
:102920000FB6F8949EBF0FBE8DBFEDB7FEB73196C0
:10293000ADB7BEB712961C930E93119780EE91E03F
:102940009383828383E890E0958384838091D40489
:102950009091D504A091D604B091D7048683978333
:10296000A087B18784E890E0938782878091E40410
:102970009091E504A091E604B091E70484879587DF
:10298000A687B7870E94E2298DB79EB740960FB6FB
:10299000F8949EBF0FBE8DBFC8010E942F051F91E6
:1029A0000F9108950F931F93282F462F86EA94E0E6
:1029B000622F0E94730486EA94E00E944B05809186
:1029C000E904282F30E0823030F4F4E0220F331F86
:1029D000FA95E1F702C02150304000D000D000D07D
:1029E000EDB7FEB7319606EA14E0ADB7BEB7129662
:1029F0001C930E93119780E091E09383828335833B
:102A000024830E94E2298DB79EB706960FB6F894EC
:102A10009EBF0FBE8DBFC8010E942F051F910F9151
:102A200008950F931F93282F462F06EA14E0C8013C
:102A3000622F0E947304C8010E944B058DB79EB798
:102A400008970FB6F8949EBF0FBE8DBFEDB7FEB7C7
:102A50003196ADB7BEB712961C930E93119782EFC5
:102A600091E0938382838FE090E0958384838091CB
:102A7000E804868317820E94E2298DB79EB70896E4
:102A80000FB6F8949EBF0FBE8DBFC8010E942F05E0
:102A90001F910F9108950F931F9306EA14E0C80148
:102AA00063E045E00E947304C8010E944B0500D01A
:102AB00000D0EDB7FEB71283018384E691E09483E2
:102AC00083830E94D129EDB7FEB71283018380E58D
:102AD00091E0948383830E94D129EDB7FEB71283DE
:102AE000018389E491E0948383830E94D129EDB727
:102AF000FEB71283018383E491E0948383830E9471
:102B0000D1290F900F900F900F90C8010E942F05B0
:102B10001F910F9108950F931F93282F462F06EAB8
:102B200014E0C801622F0E947304C8010E944B0583
:102B300000D000D0EDB7FEB7128301838BE791E0A0
:102B4000948383830E94D1290F900F900F900F9050
:102B5000C8010E942F051F910F910895EF92FF92D7
:102B60000F931F93CF93DF930E947B3120915006E8
:102B7000309151064091520650915306261737075F
:102B80004807590708F08AC10E947B316C507E4F7C
:102B90008F4F9F4F6093500670935106809352065B
:102BA0009093530606EA14E0C8010E949805C801F4
:102BB00065E043E00E947304C8010E944B0500D009
:102BC00000D0EDB7FEB7128301838BED91E09483C3
:102BD00083830E94D1290F900F900F900F908091C6
:102BE000340690913506892B31F080914B069091F7
:102BF0004C06892B81F48091E0049091E10490933C
:102C00003506809334068091E2049091E30490931A
:102C10004C0680934B062091E2043091E3044091EE
:102C20004B0650914C06C9018456904048175907ED
:102C300024F480914F068F5F08C02C593F4F241712
:102C400035072CF480914F06815080934F06809178
:102C50004F06181614F081E003C084301CF083E0A6
:102C600080934F0680914F06823009F462C0833012
:102C700009F4BEC0813009F00DC100D000D0C6EA11
:102C8000D4E0EDB7FEB7D283C18382ED91E09483A7
:102C900083830E94D129809125060F900F900F9079
:102CA0000F9080FF22C000D000D0EDB7FEB7D283D6
:102CB000C1838AEC91E0948383830E94D12980911F
:102CC000340690913506845690400F900F900F90E7
:102CD0000F902091E0043091E104281739070CF09F
:102CE000D9C0809125068E7F21C000D000D0EDB7DD
:102CF000FEB7D283C18382EC91E0948383830E94E8
:102D0000D12980913406909135068C599F4F0F90B0
:102D10000F900F900F902091E0043091E104821702
:102D200093070CF0B7C0809125068160809325063B
:102D3000B1C000D000D0C6EAD4E0EDB7FEB7D28370
:102D4000C18388EB91E0948383830E94D1290F9003
:102D50000F900F900F9080914D06882301F100D0C5
:102D600000D0EDB7FEB7D283C1838EEA91E09483A1
:102D700083830E94D1298091340690913506845630
:102D800090400F900F900F900F902091E0043091A1
:102D9000E104281739071CF510924D0620C000D019
:102DA00000D0EDB7FEB7D283C18381EA91E094836E
:102DB00083830E94D12980913406909135068C59E5
:102DC0009F4F0F900F900F900F902091E004309143
:102DD000E104821793071CF481E080934D068FE98C
:102DE00096E06BEF73E040914D060E949A3052C01E
:102DF00000D000D0A6EAEA2EA4E0FA2EEDB7FEB786
:102E0000F282E18280E991E0948383830E94D12958
:102E10008DB79EB708970FB6F8949EBF0FBE8DBFB3
:102E20000DB71EB70F5F1F4FEDB7FEB7F282E182FD
:102E300088EF91E0F8019383828360914E0670E001
:102E400080E090E00E94D93420E030E040E251E49C
:102E50000E944034F801648375838683978386E7F4
:102E600090E09187808780E290E0938782870E943C
:102E7000E2298DB79EB70C960FB6F8949EBF0FBE91
:102E80008DBF80914E0690E060E873E00E94D50C03
:102E900080934E0686EA94E00E942F05DF91CF9141
:102EA0001F910F91FF90EF9008952F923F924F92B4
:102EB0005F926F927F928F929F92AF92BF92CF92CA
:102EC000DF92EF92FF920F931F93DF93CF93CDB7D3
:102ED000DEB72B970FB6F894DEBF0FBECDBF888745
:102EE00069870E947B3120915D0630915E0640919A
:102EF0005F0650916006261737074807590708F004
:102F000069C1809161068823C9F08093AE02109256
:102F1000610680E092E090936306809362060E94CF
:102F20007B316C507E4F8F4F9F4F60935D06709347
:102F30005E0680935F069093600607C18091AE02A3
:102F4000282E33242091DC042F83009162061091F7
:102F500063063091C90439838091E9048E8390918E
:102F600054069D83E09016056090F6047090F70477
:102F70008090F8049090F90490914E064090AC0235
:102F80005090AD0280915506A82FB0E0BC83AB8372
:102F9000B0915606BA83F09015053B862A86A92E75
:102FA000BB24CC24DD24EA85FB853196FB87EA87A8
:102FB00037972CF021E030E03B872A871CC08A85B8
:102FC0009B858330910539F1843091053CF4813043
:102FD000910589F0029709F07FC015C0AA85BB85CD
:102FE000A530B10509F44EC0A530B10504F116971E
:102FF00009F072C058C0BF81B23008F06DC00DE05A
:1030000012E081E070C0E981E33009F465C00AE1B3
:1030100012E082E068C0FE81F23008F05DC02D81D0
:10302000222309F459C007E212E083E05CC031E0DA
:103030003E1598F0C601B5010E94D93420E030E079
:1030400040E251E40E9440349B01AC01C401B30151
:103050000E94393488230CF03FC004E312E083E07F
:10306000E81649F094E0E91649F0A2E0EA1641F4C6
:1030700001E412E005C00EE412E002C00BE512E02C
:1030800084E031C0EB81FC814E165F062CF5FDE932
:103090004F16FFEF5F0601F12A812223E9F408E6CB
:1030A00012E085E020C03F813230B0F481E08F151E
:1030B00098F493E0F91649F0A4E0FA1649F0B2E06A
:1030C000FB1651F405E712E005C001E812E002C06A
:1030D0000EE812E086E007C0EA85FB85E215F305FD
:1030E00009F061CF60C0109363060093620680937D
:1030F000610681E0809357060E947B3168517C4FC6
:103100008F4F9F4F60935D0670935E0680935F06BE
:10311000909360060E947B316056704F8F4F9F4F97
:103120006093590670935A0680935B0690935C06F1
:1031300080915806882321F086EA94E00E94980541
:103140001092580602C01092570606EA14E0C80111
:10315000688549850E947304C8010E944B0500D010
:1031600000D000D0EDB7FEB73196ADB7BEB712961E
:103170001C930E9311978BE992E093838283809145
:10318000620690916306958384830E94E229EDB7DD
:10319000FEB736960FB6F894FEBF0FBEEDBFC8015E
:1031A0000E942F0517C010936306009362061092C9
:1031B00061060E947B312091590630915A06409158
:1031C0005B0650915C06261737074807590708F435
:1031D000BACFBBCF2B960FB6F894DEBF0FBECDBFD4
:1031E000CF91DF911F910F91FF90EF90DF90CF90E3
:1031F000BF90AF909F908F907F906F905F904F9017
:103200003F902F900895EF92FF920F931F9380911C
:103210006406843009F056C09091DD04943008F0C3
:1032200027C180916D068917A1F190936D060E94C8
:103230007B316093690670936A0680936B06909366
:103240006C0690916D068091AF02981711F58091F0
:103250005806813091F0813018F08230B1F413C0FB
:1032600011E0109358060E947B31615375478040EE
:10327000904030F41093650608C082E080935806B1
:103280001092650602C01092580686EA94E00E94E9
:1032900098050E947B312091690630916A06409121
:1032A0006B0650916C06621B730B840B950B615D72
:1032B00077408040904008F4DBC08091DD0480932B
:1032C000AF02D6C0853029F48091A4029091A50266
:1032D00014C0863029F48091A6029091A7020DC0F7
:1032E000873029F48091A8029091A90206C0883005
:1032F00041F48091AA029091AB029093680680936A
:1033000067068091660620916706309168068823DB
:1033100009F04AC0C901895097408F5A9440C8F4B7
:103320000E947B31615375478040904020F481E0DA
:10333000809365060CC080916506882341F48091D6
:103340005706882321F486EA94E00E94980582E0DB
:1033500028C044E0203B340768F480915806882355
:1033600049F01092650686EA94E00E949805109252
:1033700058067EC0205B34402955324008F078C0A2
:1033800080915806813009F473C0809157068823D4
:1033900009F06EC01092650686EA94E00E949805D6
:1033A00081E08093580664C0215B344008F460C01B
:1033B0000E947B31615375478040904008F041C0C6
:1033C000809165068823E9F5E0906906F0906A0629
:1033D00000916B0610916C0688EE93E0A0E0B0E0DF
:1033E000E80EF91E0A1F1B1F0E947B31E616F70626
:1033F00008071907E8F581E08093650617C0109269
:10340000650686EA94E00E9498058091580682300D
:1034100019F41092580603C08F5F8093580680916C
:103420005806823018F082E0809358060E947B3163
:103430006093690670936A0680936B0690936C069E
:1034400017C0E0906906F0906A0600916B06109133
:103450006C0688EE93E0A0E0B0E0E80EF91E0A1FCB
:103460001B1F0E947B31E616F7060807190738F282
:103470001F910F91FF90EF90089580916406843022
:1034800010F00E94031980916506882319F00E94AC
:10349000AE1508958091090480FF08C060916F0403
:1034A00080916D0490E070E00E945517809158065D
:1034B000823008F0FDC1A82FB0E0FD01ED5FFB4FA9
:1034C000808185FF0BC0FD01E15EFB4F6081A35E43
:1034D000BB4F8C9190E070E00E94111580915806CE
:1034E000A82FB0E0FD01ED5FFB4F808186FF0BC090
:1034F000FD01ED5DFB4F6081AF5DBB4F8C9190E0B6
:1035000070E00E94D21480915406882309F43FC0D1
:1035100080915806A82FB0E0FD01ED5FFB4F808140
:1035200087FF0BC0FD01E95DFB4F6081AB5DBB4FC9
:103530008C9190E070E00E94801480915806A82F32
:10354000B0E0FD01EB5FFB4F808184FF0BC0FD010C
:10355000E15CFB4F6081A35CBB4F8C9190E070E01D
:103560000E94271480915806A82FB0E0FD01EB5F60
:10357000FB4F808183FF0BC0FD01E55CFB4F608149
:10358000A75CBB4F8C9190E070E00E94101480917A
:103590005806A82FB0E0FD01E95FFB4F808187FF4F
:1035A0000BC0FD01E95AFB4F6081AB5ABB4F8C91B8
:1035B00090E070E00E94B71380915806A82FB0E009
:1035C000FD01E75FFB4F808183FF0BC0FD01E958E0
:1035D000FB4F6081AB58BB4F8C9190E070E00E9434
:1035E000221280915406882309F46EC08091E90468
:1035F000823008F469C080915806A82FB0E0FD0120
:10360000E55FFB4F808182FF0BC0FD01ED57FB4F53
:103610006081AF57BB4F8C9190E070E00E946812C0
:1036200080915806A82FB0E0FD01E95FFB4F808133
:1036300082FF0BC0FD01ED5AFB4F6081AF5ABB4FBB
:103640008C9190E070E00E94601380915806A82F42
:10365000B0E0FD01E95FFB4F808183FF0BC0FD01FE
:10366000E55AFB4F6081A75ABB4F8C9190E070E008
:103670000E94091380915806A82FB0E0FD01EB5F6E
:10368000FB4F808181FF0BC0FD01ED5CFB4F608132
:10369000AF5CBB4F8C9190E070E00E94E011809194
:1036A0005806A82FB0E0FD01EB5FFB4F808180FF43
:1036B0000BC0FD01E15DFB4F6081A35DBB4F8C91B1
:1036C00090E070E00E949E1180915806A82FB0E013
:1036D000FD01E75FFB4F808186FF0BC0FD01E158D4
:1036E000FB4F6081A358BB4F8C9190E070E00E942B
:1036F0005E1180915806A82FB0E0FD01ED5FFB4FF1
:10370000808182FF0BC0FD01E95EFB4F6081AB5EF3
:10371000BB4F8C9190E070E00E941E118091580682
:10372000A82FB0E0FD01ED5FFB4F808181FF0BC052
:10373000FD01ED5EFB4F6081AF5EBB4F8C9190E071
:1037400070E00E94DE1080915806A82FB0E0FD01C5
:10375000E95FFB4F808184FF0BC0FD01ED59FB4FFA
:103760006081AF59BB4F8C9190E070E00E949E1039
:1037700080915806A82FB0E0FD01E95FFB4F8081E2
:1037800085FF0BC0FD01E959FB4F6081AB59BB4F71
:103790008C9190E070E00E94061080915806A82F4E
:1037A000B0E0FD01ED5FFB4F808183FF0BC0FD01A9
:1037B000E55EFB4F6081A75EBB4F8C9190E070E0AF
:1037C0000E94C00F80915806A82FB0E0FD01E95F6C
:1037D000FB4F808180FF0BC0FD01E15BFB4F6081EF
:1037E000A35BBB4F8C9190E070E00E946B0F8091C7
:1037F0005806A82FB0E0FD01ED5FFB4F808184FFEC
:103800000BC0FD01E55DFB4F6081A75DBB4F8C9157
:1038100090E070E00E942B0F80915806A82FB0E036
:10382000FD01E55FFB4F808181FF18C080914D064F
:10383000FD01EB57FB4F813049F4A957BB4F6C9109
:10384000808190E070E00E940F0E08C0A957BB4F26
:103850006C91808190E070E00E94620E8091580629
:10386000A82FB0E0FD01EB5FFB4F808187FF0BC00D
:10387000FD01E55BFB4F6081A75BBB4F8C9190E046
:1038800070E00E948C0D80915806A82FB0E0FD01D9
:10389000E95FFB4F808186FF0BC0FD01E559FB4FBF
:1038A0006081A759BB4F8C9190E070E00E94310D70
:1038B000089586EA94E00E9498050E944B150E94A4
:1038C0000A0A0895CF93DF93EC0186EA94E00E9400
:1038D0006F04C817D9073CF086EA94E00E9464049C
:1038E000892B09F42397CE01DF91CF910895EF92B0
:1038F000FF920F931F93CF93DF930091580610E030
:103900008AEF90E0089F7001099FF00C189FF00C5F
:103910001124C7010E94EF0AF801ED5FFB4F8823D5
:1039200019F08081816002C080818E7F80838091C8
:103930005806C82FD0E0C70102960E94EF0AC35F65
:10394000DB4F888380915806C82FD0E0C7010496CA
:103950000E94EF0A90E00E94621CC15FDB4F8883E7
:103960000091580610E0C70188569F4F0E94EF0A49
:10397000F801ED5FFB4F882319F08081806102C060
:1039800080818F7E808380915806C82FD0E0C70148
:1039900086569F4F0E94EF0AC75DDB4F8883809158
:1039A0005806C82FD0E0C70184569F4F0E94EF0AE7
:1039B00090E00E94621CC55DDB4F88830091580631
:1039C00010E0C70106960E94EF0AF801ED5FFB4F79
:1039D000882319F08081826002C080818D7F80837E
:1039E00080915806C82FD0E0C70108960E94EF0AC0
:1039F000CF5EDB4F888380915806C82FD0E0C70187
:103A00000A960E94EF0A90E00E94621CCD5EDB4F96
:103A100088830091580610E0C7010C960E94EF0AB7
:103A2000F801ED5FFB4F882319F08081846002C0AC
:103A300080818B7F808380915806C82FD0E0C7019A
:103A40000E960E94EF0ACB5EDB4F8883809158066A
:103A5000C82FD0E0C70140960E94EF0A90E00E9474
:103A6000621CC95EDB4F88830091580610E0C701D5
:103A700042960E94EF0AF801ED5FFB4F882319F090
:103A80008081886002C08081877F80838091580612
:103A9000C82FD0E0C70144960E94EF0AC75EDB4FF3
:103AA000888380915806C82FD0E0C70146960E94AF
:103AB000EF0A90E00E94621CC55EDB4F8883009194
:103AC000580610E0C7014E960E94EF0AF801ED5F1C
:103AD000FB4F882319F08081806202C080818F7D36
:103AE000808380915806C82FD0E0C70180960E943D
:103AF000EF0AC35EDB4F888380915806C82FD0E061
:103B0000C70182960E94EF0A90E00E94621CC15E8B
:103B1000DB4F88830091580610E0C70184960E940D
:103B2000EF0AF801ED5FFB4F882319F08081806474
:103B300002C080818F7B808380915806C82FD0E09F
:103B4000C70186960E94EF0ACF5DDB4F8883809184
:103B50005806C82FD0E0C70188960E94EF0A90E06F
:103B60000E94621CCD5DDB4F88830091580610E0F7
:103B7000C7018A960E94EF0AF801ED5FFB4F882388
:103B800019F08081806802C080818F778083809166
:103B90005806C82FD0E0C7018C960E94EF0ACB5D73
:103BA000DB4F888380915806C82FD0E0C7018E96DE
:103BB0000E94EF0A90E00E94621CC95DDB4F88837F
:103BC0000091580610E0C701C0960E94EF0AF80164
:103BD000EB5FFB4F882319F08081816002C08081F8
:103BE0008E7F808380915806C82FD0E0C701C2968F
:103BF0000E94EF0AC35DDB4F888380915806C82F6F
:103C0000D0E0C701C4960E94EF0A90E00E94621CB7
:103C1000C15DDB4F88830091580610E0C701C6964E
:103C20000E94EF0AF801EB5FFB4F882319F08081B7
:103C3000826002C080818D7F808380915806C82F6A
:103C4000D0E0C701C8960E94EF0ACF5CDB4F8883A3
:103C500080915806C82FD0E0C701CA960E94EF0A8B
:103C600090E00E94621CCD5CDB4F88830091580677
:103C700010E0C701CC960E94EF0AF801EB5FFB4F02
:103C8000882319F08081846002C080818B7F8083CB
:103C900080915806C82FD0E0C701CE960E94EF0A47
:103CA000CB5CDB4F888380915806C82FD0E0C701DA
:103CB000805C9F4F0E94EF0A90E00E94621CC95CEA
:103CC000DB4F88830091580610E0C701885B9F4F47
:103CD0000E94EF0AF801EB5FFB4F882319F0808107
:103CE000806102C080818F7E808380915806C82FBA
:103CF000D0E0C701865B9F4F0E94EF0AC35CDB4F99
:103D0000888380915806C82FD0E0C701845B9F4FFD
:103D10000E94EF0A90E00E94621CC15CDB4F888326
:103D20000091580610E0C7018E5B9F4F0E94EF0A7A
:103D3000F801EB5FFB4F882319F08081886002C097
:103D40008081877F808380915806C82FD0E0C7018B
:103D50008C5B9F4F0E94EF0AC75CDB4F888380918A
:103D60005806C82FD0E0C7018A5B9F4F0E94EF0A18
:103D700090E00E94621CC55CDB4F8883009158066E
:103D800010E0C701805B9F4F0E94EF0AF801EB5FD4
:103D9000FB4F882319F08081806202C080818F7D73
:103DA000808380915806C82FD0E0C7018E5A9F4F5C
:103DB0000E94EF0ACF5BDB4F888380915806C82FA3
:103DC000D0E0C7018C5A9F4F0E94EF0A90E00E94FA
:103DD000621CCD5BDB4F88830091580610E0C70161
:103DE0008A5A9F4F0E94EF0AF801EB5FFB4F88232E
:103DF00019F08081806402C080818F7B80838091F4
:103E00005806C82FD0E0C701885A9F4F0E94EF0A7A
:103E1000CB5BDB4F888380915806C82FD0E0C70169
:103E2000865A9F4F0E94EF0A90E00E94621CC95B75
:103E3000DB4F88830091580610E0C70182569F4FE0
:103E40000E94EF0AF801EB5FFB4F882319F0808195
:103E5000806802C080818F77808380915806C82F48
:103E6000D0E0C70180569F4F0E94EF0AC75BDB4F2F
:103E7000888380915806C82FD0E0C7018E559F4F88
:103E80000E94EF0A90E00E94621CC55BDB4F8883B2
:103E90000091580610E0C7018E599F4F0E94EF0A0B
:103EA000F801E95FFB4F882319F08081816002C02F
:103EB00080818E7F808380915806C82FD0E0C70113
:103EC0008C599F4F0E94EF0AC35BDB4F8883809120
:103ED0005806C82FD0E0C7018A599F4F0E94EF0AA9
:103EE00090E00E94621CC15BDB4F88830091580602
:103EF00010E0C70182599F4F0E94EF0AF801E95F65
:103F0000FB4F882319F08081846002C080818B7F01
:103F1000808380915806C82FD0E0C70180599F4FF9
:103F20000E94EF0ACF5ADB4F888380915806C82F32
:103F3000D0E0C7018E589F4F0E94EF0A90E00E9488
:103F4000621CCD5ADB4F88830091580610E0C701F0
:103F500084579F4F0E94EF0AF801E95FFB4F8823C7
:103F600019F08081806802C080818F778083809182
:103F70005806C82FD0E0C70182579F4F0E94EF0A12
:103F8000CB5ADB4F888380915806C82FD0E0C701F9
:103F900080579F4F0E94EF0A90E00E94621CC95A0E
:103FA000DB4F88830091580610E0C7018E569F4F63
:103FB0000E94EF0AF801E95FFB4F882319F0808126
:103FC000826002C080818D7F808380915806C82FD7
:103FD000D0E0C7018C569F4F0E94EF0AC35ADB4FB7
:103FE000888380915806C82FD0E0C7018A569F4F1A
:103FF0000E94EF0A90E00E94621CC15ADB4F888346
:104000000091580610E0C7018C589F4F0E94EF0A9C
:10401000F801E95FFB4F882319F08081886002C0B6
:104020008081877F808380915806C82FD0E0C701A8
:104030008A589F4F0E94EF0AC75ADB4F88838091AE
:104040005806C82FD0E0C70188589F4F0E94EF0A3A
:1040500090E00E94621CC55ADB4F8883009158068D
:1040600010E0C70186589F4F0E94EF0AF801E95FF0
:10407000FB4F882319F08081806102C080818F7E90
:10408000808380915806C82FD0E0C70184589F4F85
:104090000E94EF0ACF59DB4F888380915806C82FC2
:1040A000D0E0C70182589F4F0E94EF0A90E00E9423
:1040B000621CCD59DB4F88830091580610E0C70180
:1040C00080589F4F0E94EF0AF801E95FFB4F882359
:1040D00019F08081806202C080818F7D8083809111
:1040E0005806C82FD0E0C7018E579F4F0E94EF0A95
:1040F000CB59DB4F888380915806C82FD0E0C70189
:104100008C579F4F0E94EF0A90E00E94621CC95991
:10411000DB4F88830091580610E0C7018A579F4FF4
:104120000E94EF0AF801E95FFB4F882319F08081B4
:10413000806402C080818F7B808380915806C82F65
:10414000D0E0C70188579F4F0E94EF0AC759DB4F45
:10415000888380915806C82FD0E0C70186579F4FAB
:104160000E94EF0A90E00E94621CC559DB4F8883D1
:104170000091580610E0C7018C559F4F0E94EF0A2E
:10418000F801E75FFB4F882319F08081816002C04E
:1041900080818E7F808380915806C82FD0E0C70130
:1041A0008A559F4F0E94EF0AC359DB4F8883809145
:1041B0005806C82FD0E0C70188559F4F0E94EF0ACC
:1041C00090E00E94621CC159DB4F88830091580621
:1041D00010E0C70180559F4F0E94EF0AF801E75F8A
:1041E000FB4F882319F08081846002C080818B7F1F
:1041F000808380915806C82FD0E0C7018E549F4F0E
:104200000E94EF0ACF58DB4F888380915806C82F51
:10421000D0E0C7018C549F4F0E94EF0A90E00E94AB
:10422000621CCD58DB4F88830091580610E0C7010F
:104230008A549F4F0E94EF0AF801E75FFB4F8823E3
:1042400019F08081886002C08081877F808380919F
:104250005806C82FD0E0C70188549F4F0E94EF0A2C
:10426000CB58DB4F888380915806C82FD0E0C70118
:1042700086549F4F0E94EF0A90E00E94621CC9582A
:10428000DB4F88830091580610E0C70184549F4F8C
:104290000E94EF0AF801E75FFB4F882319F0808145
:1042A000806102C080818F7E808380915806C82FF4
:1042B000D0E0C70182549F4F0E94EF0AC758DB4FDE
:1042C000888380915806C82FD0E0C70180549F4F43
:1042D0000E94EF0A90E00E94621CC558DB4F888361
:1042E0000091580610E0C701845A9F4F0E94EF0AC0
:1042F000F801E75FFB4F882319F08081806402C0DA
:1043000080818F7B808380915806C82FD0E0C701C1
:10431000825A9F4F0E94EF0AC358DB4F88838091D7
:104320005806C82FD0E0C701805A9F4F0E94EF0A5D
:1043300090E00E94621CC158DB4F888300915806B0
:1043400010E0C70180529F4F0E94EF0AF801E55F1D
:10435000FB4F882319F08081846002C080818B7FAD
:10436000808380915806C82FD0E0C7018E519F4F9F
:104370000E94EF0ACF57DB4F888380915806C82FE1
:10438000D0E0C7018C519F4F0E94EF0A90E00E943D
:10439000621CCD57DB4F88830091580610E0C7019F
:1043A0008C529F4F0E94EF0AF801E55FFB4F882374
:1043B00019F08081826002C080818D7F808380912E
:1043C0005806C82FD0E0C7018A529F4F0E94EF0ABB
:1043D000CB57DB4F888380915806C82FD0E0C701A8
:1043E00088529F4F0E94EF0A90E00E94621CC957BA
:1043F000DB4F8883DF91CF911F910F91FF90EF905A
:1044000008954F925F927F928F929F92AF92BF9248
:10441000CF92DF92EF92FF920F931F93DF93CF9390
:10442000CDB7DEB7C854D0400FB6F894DEBF0FBE8C
:10443000CDBF06EA14E0C8010E949805C80166E0F5
:1044400049E00E947304C8010E944B0500D000D0CF
:10445000EDB7FEB71283018386E092E094838383F5
:104460000E94D1290F900F900F900F90C8010E94C9
:104470002F0500D000D009E814E0EDB7FEB7128395
:10448000018386EF91E0948383830E94D1294BEED0
:10449000442E41E0542EEE24FF24CC24DD240F9042
:1044A0000F900F900F90702E012F39E0A32EB12C9A
:1044B000AC0EBD1E4E010894811C911C89E894E04D
:1044C0000E94852A982F8D3031F08D30DCF1805399
:1044D0008230C0F530C01830A1F59981892F805302
:1044E000823078F5913311F490E801C090E08A8130
:1044F000813309F4905C8B81813309F4905E8C8167
:10450000813309F4905F8D81813309F4985F8E8146
:10451000813309F49C5F8F81813309F49E5F888524
:10452000813309F49F5FF501EE0DFF1D9083089420
:10453000E11CF11C06C0F401E10FF11D90831F5F27
:1045400001C010E0F0E4EF16F104C9F486EA94E04B
:10455000B601A5010E9483040894C11CD11C00D09F
:1045600000D0EDB7FEB771820283548243820E946D
:10457000D129EE24FF240F900F900F900F90FFEFA2
:10458000CF16D10409F00CF499CFC85BDF4F0FB6FA
:10459000F894DEBF0FBECDBFCF91DF911F910F9179
:1045A000FF90EF90DF90CF90BF90AF909F908F9053
:1045B0007F905F904F900895DF92EF92FF920F935C
:1045C0001F93DF93CF93CDB7DEB72A970FB6F8943A
:1045D000DEBF0FBECDBF63E0E62EF12CEC0EFD1E5C
:1045E00053E0D52EC9C30E947B3160527E44804087
:1045F0009040C8F40E947B316958734180409040DC
:1046000090F01A3011F01D3031F4809121068F5F47
:104610008093210602C010922106809121068330EA
:1046200011F40E940122812F67E175E00E94F506D6
:10463000882311F400E09AC380911B0590911C051A
:10464000A0911D05B0911E058A3747EC940749EDEE
:10465000A4074BE7B40709F477C38B3757EC9507EA
:1046600059EDA5075BE7B50708F0D4C0823DE2EC41
:104670009E07E2E8AE07EEE1BE0709F403C2833D00
:10468000F2EC9F07F2E8AF07FEE1BF0708F061C058
:1046900088392CE292072AE1A20726E1B20709F441
:1046A000F1C189393CE293073AE1A30736E1B30748
:1046B00040F586314AEA940747E3A4074BE0B40784
:1046C00009F4D7C187315AEA950757E3A5075BE09C
:1046D000B50738F48E5F9B4CA74CB94009F03CC33A
:1046E00033C38430FAE99F07F7EDAF07FEE0BF0759
:1046F00009F4BFC18259934AAC4EB44109F02CC3AE
:10470000B8C18E3C38E4930737E5A3073AE1B30715
:1047100009F404C28F3C48E4940747E5A4074AE142
:10472000B40738F480559F4DAD4EB84109F014C31D
:10473000E0C28437EBEE9E07EAE7AE07EBE1BE0787
:1047400009F497C184549B4DA047BD4109F004C3AF
:10475000FBC2863A2EE0920722E1A20728E4B207C4
:1047600009F492C2873A3EE0930732E1A30738E4A6
:10477000B30740F5823543E2940746E9A40746E2D1
:10478000B40709F448C2833553E2950756E9A507F3
:1047900056E2B50738F488529E45A24DB44209F05E
:1047A000DBC267C1863EF5ED9F07FAEDAF07F3E385
:1047B000BF0709F40CC1885F9C4AAE4EB44309F0B0
:1047C000CBC2C2C2823E35E593073CE9A30736E679
:1047D000B30709F480C2833E45E594074CE9A4077A
:1047E00046E6B40738F48855964BAD4FBA4409F005
:1047F000B3C261C28C3EE9E39E07E6E7AE07EBE693
:10480000BE0709F4A1C280569B4DAB43BE4609F0DA
:10481000A3C22FC18A3B24E8920725E2A2072EEB10
:10482000B20709F458C28B3B34E8930735E2A3077B
:104830003EEBB30708F061C08E3742E194074AE6C9
:10484000A4074BE9B40709F414C18F3752E1950767
:104850005AE6A5075BE9B50740F58235EAEE9E0703
:10486000E0E8AE07EAE8BE0709F403C18335FAEED3
:104870009F07F0E8AF07FAE8BF0738F4865E964A6C
:10488000A642BD4709F068C249C18C3835E8930794
:1048900037EAA30738E9B30709F440C18A569E42B4
:1048A000A246B94909F058C2EFC180325EE49507CB
:1048B00059EAA50751EBB50709F40DC28132EEE4C0
:1048C0009E07E9EAAE07E1EBBE0738F48A57964F38
:1048D000A14FBD4909F040C221C18A3827EF920794
:1048E00027ECA20728EBB20709F4CCC0845A904009
:1048F000AB49BA4B09F030C227C2843649ED940760
:1049000040EEA40747EDB40709F461C0853659EDC0
:10491000950750EEA50757EDB50740F58038E4E759
:104920009E07E0E1AE07E4ECBE0709F4ABC08138B6
:10493000F4E79F07F0E1AF07F4ECBF0738F48C56BB
:104940009846A344B24C09F007C255C184353DE2F4
:1049500093073FEFA30735ECB30709F48AC08659E4
:104960009543A840B24D09F0F7C155C18E345DE5BD
:1049700095075EE3A50753EEB50709F47AC08F34B7
:10498000EDE59E07EEE3AE07E3EEBE0780F4843765
:10499000F7E39F07F4EDAF07FEEDBF0709F49BC1F6
:1049A000865B9342A34AB24E09F0D6C1B7C08239A2
:1049B00030E7930736E8A3073BEFB30709F4C4C118
:1049C000825F9D4EA442BD4F09F0C6C18DC10E94B9
:1049D0007B316093CA047093CB048093CC04909392
:1049E000CD04D092C90487E195E060E170E00E94B7
:1049F000C9080E94A8347093CF046093CE0487E165
:104A000095E064E170E00E94C9080E94A8347093A8
:104A1000D1046093D00487E195E068E170E00E94E2
:104A2000C9080E94A8348B017093D3046093D20408
:104A30006091D4047091D5048091D6049091D704EC
:104A400020E030E040E050E00E943934882379F4DF
:104A5000B801882777FD8095982F0E94DB346093FA
:104A6000D8047093D9048093DA049093DB0401E0B6
:104A700074C1809121058093DC048091220580938C
:104A8000DD046AC187E195E060E070E00E94C9083A
:104A900020E030E048EC52E40E940E360E94A83438
:104AA0007093DF046093DE04693C710520F010927E
:104AB000DF041092DE0480913B0590913C059093B9
:104AC000E1048093E00480913D0590913E05909330
:104AD000E3048093E2048091410590914205909314
:104AE000A5028093A402809145059091460590937C
:104AF000A7028093A6028091470590914805909364
:104B0000A9028093A8028091490590914A059A8351
:104B100089839093AB028093AA021EC16091210504
:104B20007091220580912305909124050E94DB3429
:104B300020E836E948E15BE40E9440346093D40405
:104B40007093D5048093D6049093D7046091250583
:104B5000709126058091270590912805D7016C93C7
:104B600011967C93119712968C93129713969C939F
:104B70000E94DB3420E836E948E15BE40E944034DF
:104B80006093E4047093E5048093E6049093E70453
:104B9000809146058093E804809145058093E9045F
:104BA00087E195E060E170E00E94C9086093D80455
:104BB0007093D9048093DA049093DB0487E195E045
:104BC00068E070E00E94C9086093EA047093EB0407
:104BD0008093EC049093ED0487E195E064E170E04C
:104BE0000E94C9086093EE047093EF048093F00470
:104BF0009093F104B1C087E195E068E070E00E9415
:104C0000C90890586093F2047093F3048093F404FD
:104C10009093F504A1C087E195E060E070E00E9408
:104C2000C9086093F6047093F7048093F804909396
:104C3000F90487E195E064E070E00E94C90820E093
:104C400030E048EC52E40E940E360E94A834709383
:104C5000FB046093FA0487E195E064E170E00E9450
:104C6000C9080E94A8347093FD046093FC0487E196
:104C700095E068E170E00E94C9080E94A834709332
:104C8000FF046093FE0468C087E195E064E070E093
:104C90000E94C9080E94A834882777FD8095982F24
:104CA0000E94DB3460930005709301058093020538
:104CB0009093030551C087E195E068E070E00E94A1
:104CC000C9080E94A834709561957F4F70930505BF
:104CD0006093040541C08091810580930605809111
:104CE00082058093070538C08091210580930805CF
:104CF00033C087E195E060E070E00E94C9086093EE
:104D0000090570930A0580930B0590930C0587E1C4
:104D100095E064E070E00E94C90860930D0570930F
:104D20000E0580930F059093100587E195E068E0EC
:104D300070E00E94C908609311057093120580937A
:104D400013059093140508C080912D0580931505D7
:104D5000809132058093160500E08091180582321B
:104D600029F487E195E063E20E94E1098EEB90E08F
:104D70000E94E231002331F589E894E00E94552A2F
:104D800018161906F4F489E894E00E94852A182F71
:104D90008091C904882309F046CC25CC1092C9041F
:104DA00001E0802F90E02A960FB6F894DEBF0FBE88
:104DB000CDBFCF91DF911F910F91FF90EF90DF90CA
:104DC000089500E02091CA043091CB044091CC04B6
:104DD0005091CD04205F384D4F4F5F4F2F83388760
:104DE00049875A870E947B312F81388549855A85AA
:104DF000261737074807590788F2D3CFEF92FF925B
:104E00000F931F9380915606882351F083E00E94F0
:104E1000173364E070E00E944837609326063CC078
:104E200083E00E941733AA2797FDA095BA2FBC01F3
:104E3000CD010E94DB342DEC3CEC4CE45EE30E949F
:104E40000E3620E030E040E85EE30E940E367B0143
:104E50008C016091260670E0882777FD8095982F59
:104E60000E94DB342DEC3CEC4CE45FE30E940E36F8
:104E70009B01AC01C801B7010E9473330E94AD349D
:104E800020917106621730F030917006262F361788
:104E900008F4232F209326061F910F91FF90EF9087
:104EA000089583E00E94143308951F93CF93DF93F6
:104EB00085E090E06CE070E00E948B1568EE73E096
:104EC00080E090E00E94893189E894E00E94D22A33
:104ED000C0E0D0E010E0CE016DE171E00E94483703
:104EE000892BA9F41F5E86EA94E0612F4CE00E94B2
:104EF000730486EA94E00E944B0586EA94E06EEE25
:104F00000E947B0586EA94E00E942F05105161E023
:104F100070E080E090E00E948931219687E0C13DF9
:104F2000D807C9F6DF91CF911F91089586E061E01F
:104F30000E94C03208950F931F9386E061E00E94A3
:104F4000813209E814E0C80140E051EE60E070E011
:104F50000E94F3291093A1060093A0060E949627B1
:104F600086EA94E00E94D1050E94591C64EF71E02A
:104F700080E090E00E94893183EF93E00E94EF0A85
:104F8000813011F00E94000D0E94600A10925806B4
:104F900007C00E94771C809158068F5F8093580647
:104FA000809158068230A8F3109258060E94552727
:104FB0000E94512788EB94E06CE679E224E630E029
:104FC00040E050E000E00E94A63086EA94E00E94B3
:104FD000980588EB94E00E940C311F910F91089581
:104FE0002F923F924F925F926F927F928F929F92F9
:104FF000AF92BF92CF92DF92EF92FF920F931F93E7
:10500000DF93CF9300D000D0CDB7DEB780915406A8
:10501000882309F4E1C0E0907906F0907A060091C7
:105020007B0610917C06C801B7019F7725E33AEF14
:105030004EE85CE30E940E360E943D3469837A8319
:105040008B839C83C801B7012091D4043091D5048F
:105050004091D6045091D7040E9472331B012C0159
:105060009F7720EC3BE649ED57E40E940E365B014A
:105070006C0160917D0670917E0680917F06909113
:1050800080062091E4043091E5044091E6045091BB
:10509000E7040E9472333B014C019F7720EC3BE612
:1050A00049ED57E40E940E3629813A814B815C819B
:1050B0000E940E367B018C01C601B501A601950147
:1050C0000E940E365B016C01C801B701A80197016F
:1050D0000E940E369B01AC01C601B5010E947333DC
:1050E0000E9495360E94A834609347067093480644
:1050F0008093490690934A0660E070E080E89FE361
:1051000029813A814B815C810E9440349B01AC0132
:10511000C201B1010E940E3697FA909497F89094CC
:10512000A40193010E94E63320EE3EE245E652E4FC
:105130000E940E3620E030E044EB52E40E947333CC
:105140000E94A8349B01AC0197FF04C028593E4F30
:105150004F4F5F4FCA01B901645B7040804090407F
:1051600097FF06C0CA01B9016C547F4F8F4F9F4F04
:105170000E94DB342091D8043091D9044091DA04A4
:105180005091DB040E9472330E94A83497FF04C040
:1051900068597E4F8F4F9F4F0E94DB3420E030E0F4
:1051A00044EB53E40E94403420E030E040E851E416
:1051B0000E940E360E94713620E030E040E85FE346
:1051C0000E9473330E94AD3460934606613108F447
:1051D0006CC01092460669C08091E904823008F4E0
:1051E00064C08091E804853008F45FC0A090810617
:1051F0008DE18A1508F459C0E090EA04F090EB04C0
:105200000091EC041091ED04609182067091830688
:105210008091840690918506A80197010E947233BF
:105220009F7720E030E040E05FE30E9403361816ED
:105230005CF410928106E0928206F092830600935D
:1052400084061093850631C08A2D8F5F8093810676
:105250008E3159F58091D4049091D504A091D60453
:10526000B091D7048093790690937A06A0937B0639
:10527000B0937C068091E4049091E504A091E6044B
:10528000B091E70480937D0690937E06A0937F06FD
:10529000B0938006E0928606F09287060093880617
:1052A0001093890681E0809354060F900F900F9021
:1052B0000F90CF91DF911F910F91FF90EF90DF90B2
:1052C000CF90BF90AF909F908F907F906F905F90A6
:1052D0004F903F902F900895CF92DF92EF92FF92E0
:1052E0000F931F930E94FE2680912606282F30E000
:1052F0003093AD022093AC0280915606882359F575
:105300000091710610E0201B310BB901882777FD51
:105310008095982F0E94DB346B017C0160917006B0
:1053200070E0601B710B882777FD8095982F0E9495
:10533000DB349B01AC01C701B6010E94403420E080
:1053400030E048EC52E40E940E360E94A83470937C
:10535000AD026093AC02809108058093AC0210927C
:10536000AD020E9452080E94F50A86EA94E00E946B
:10537000F0270E943D1A1F910F91FF90EF90DF9050
:10538000CF9008950E94DC22892B19F00E946C298D
:10539000089588EB94E00E94F43008958FEF9FE722
:1053A0000895DF93CF93CDB7DEB7FE0139968D8197
:1053B0009E8161E04F8158859F010E94722CCF91A0
:1053C000DF910895DF93CF93CDB7DEB7FE01399615
:1053D0008D819E8160E04F8158859F010E94722CD3
:1053E000CF91DF9108950F931F93DC01ED91FC9114
:1053F0000288F389E02D20E030E000E010E009951C
:105400001F910F9108958F92AF92CF92EF92FF92DA
:105410000F931F93DF93CF93CDB7DEB7FC011382B9
:10542000128288EE93E0A0E0B0E084839583A683A7
:10543000B7838BEE93E091838083558744873787CA
:105440002687118B008BF38AE28AC48AA58A868A12
:1054500070E0CB0123E0880F991F2A95E1F79C01AA
:105460002257394F308F278B8A56994F928F818FD1
:1054700081E090E002C0880F991F6A95E2F72091C1
:105480009E06282B20939E06CF0140E051EE60E05F
:1054900070E00E94F329CF91DF911F910F91FF904F
:1054A000EF90CF90AF908F900895FC01838D88236B
:1054B00019F42FEF3FEF0DC00788F08DE02D20810C
:1054C000318182819381281B390B84819581282326
:1054D0003923C9010895FC01838D882319F42FEF26
:1054E0003FEF11C0018CF28DE02D2081318182814E
:1054F0009381281B390B2095309584819581282331
:1055000039232F5F3F4FC9010895FC01838D882304
:1055100061F0A789B08D2D913C91119712968D91D4
:105520009C9113972817390721F44FEF5FEFCA01B9
:10553000089512968D919C9113971696ED91FC917A
:105540001797E80FF91F408112968D919C91139740
:10555000019614962D913C911597822393231396CF
:105560009C938E93129750E0E2CFFC01838D8823A9
:1055700051F00788F08DE02D208131818281938167
:105580002817390721F42FEF3FEFC90108958281D1
:1055900093810680F781E02DE80FF91F8081282F85
:1055A00030E0F3CFDC015796ED91FC915897828162
:1055B0009381918380835996ED91FC915A978081D4
:1055C0009181938382830895DC015B968C915B9734
:1055D0008823A9F15996ED91FC915A972081318148
:1055E0002F5F3F4F84819581282339235C968C91CE
:1055F0005C97882329F08281938128173907F9F075
:105600008281938128173907D9F38081918106809F
:10561000F781E02DE80FF91F60835996ED91FC9119
:105620005A97318320835296ED91FC915397808154
:1056300056969C91892B808321E030E002C020E0C7
:1056400030E0C9010895CF93DF93EC011B821A82E9
:105650008A819B81998388831D821C828E819F8190
:10566000009721F00E94C5031F821E82DF91CF9117
:1056700008950F931F938C01DC015296ED91FC91DC
:105680005397208156968C91569755969C91559795
:10569000892B80958223808357968D919C91589772
:1056A0000E94232BF801818D928D0E94232BD8011B
:1056B0005B961C921F910F9108950F931F93CF93A8
:1056C000DF938C01FC01138212828281938191838A
:1056D000808341E0A1E0B0E001C04F5FFD01042EF6
:1056E00002C0EE0FFF1F0A94E2F79B0182E06130D7
:1056F000780710F020E032E0E217F30770F3C1E022
:10570000D0E002C0CC0FDD1F4A95E2F72197F801E7
:10571000268137812115310541F0848195818C17CF
:105720009D0789F0C9010E94C503F801D583C48390
:10573000CE0101960E941B039C01F801978386838A
:1057400080E0232B09F081E0DF91CF911F910F9131
:105750000895AF92BF92CF92DF92EF92FF920F9394
:105760001F93CF93DF937C015A016B01E901DC01A8
:105770005B968C915B978823F1F02115310539F404
:105780005796ED91FC915897C481D58121960115CA
:10579000110549F4D7015996ED91FC915A9704816E
:1057A00015810F5F1F4FD701ED91FC910088F189A2
:1057B000E02DC7010995F7018789908D209711F495
:1057C000C0E8D0E0BE010E945D2B882381F0D701A4
:1057D00059968D919C915A970115110511F400E18C
:1057E00010E0B8010E945D2B882309F04DC0D7015D
:1057F000ED91FC910088F189E02DC701099567C002
:10580000D7015096ED91FC915197B0E0AB16B1EEF7
:10581000BB06B0E0CB06B0E0DB0609F454C081E083
:1058200090E0D70154960C9002C0880F991F0A94FB
:10583000E2F7808360E079E08DE390E0A6019501D6
:105840000E947D372150304040405040CA01B9018C
:1058500022E030E040E050E00E947D37D7011C9606
:10586000ED91FC911D9730831E96ED91FC911F9751
:105870002083D7015296ED91FC91539780815596E4
:105880009C91892B808323C0D7015996ED91FC917F
:105890005A971382128282819381918380835796D3
:1058A000ED91FC91589713821282828193819183AA
:1058B000808381E05B968C931A141B041C041D04E6
:1058C0000CF49ECFD6CF108220E130E0C7CFDF911D
:1058D000CF911F910F91FF90EF90DF90CF90BF90ED
:1058E000AF9008952F923F924F925F926F927F9266
:1058F0008F929F92AF92BF92CF92DF92EF92FF92E0
:105900000F931F93DF93CF93CDB7DEB764970FB696
:10591000F894DEBF0FBECDBF3C01688B5A8B498B1C
:1059200069011C01AE014F5F5F4F5C8B4B8BE989B6
:10593000FA89488940FD659140FF6191FA8BE98BB6
:10594000662309F4D7C3653249F440FD859140FFD1
:105950008191FA8BE98B8532B1F40CC06A3051F435
:10596000D301ED91FC910190F081E02DC1016DE03A
:1059700009956AE0D301ED91FC910190F081E02D51
:10598000C1010995D4CF982F10E0882499241032B2
:10599000B0F49B3269F09C3228F4903251F093328B
:1059A00071F40BC09D3239F0903349F4116028C076
:1059B0001260146025C0186023C0106121C017FD5B
:1059C0002BC0892F80538A3078F416FF06C0BAE0C6
:1059D0009B9E902C1124980E13C0EAE08E9E802C82
:1059E0001124880E10620CC09E3221F416FD82C371
:1059F000106406C09C3611F4106802C0983661F439
:105A0000E989FA89488940FD959140FF9191FA8B87
:105A1000E98B992309F0BBCF892F8554833020F47B
:105A2000812F8061905E07C0892F8556833008F0F2
:105A3000E6C1812F8F7E86FD02C076E0972E6FE350
:105A4000F62EF822953619F450E4F52A07C096365A
:105A500019F480E8F82A02C091109A94F7FE0BC05E
:105A60009BE3991520F427E05CE3B52E0DC0B92C1B
:105A7000B39427E009C0A7E0A91520F447E0942ECD
:105A800027E001C0292DBB24F6013496FD87EC8761
:105A9000D6016D917D918D919C91AE014F5F5F4FCD
:105AA0000B2D0E9443026C010981E02FF0E0FF877B
:105AB000EE8700FF05C0FE85F3FD02C01DE209C0B0
:105AC000F1FE02C01BE205C0F2FC02C010E001C002
:105AD00010E28E859F858C709070892B09F444C0EC
:105AE000112311F483E001C084E0881510F08824AC
:105AF0000EC0881AF3FC0BC0D301ED91FC9101900C
:105B0000F081E02DC10160E209958A94A9F7112383
:105B100049F0D301ED91FC910190F081E02DC1019C
:105B2000612F0995BE85B3FF03C00FE013E012C0DB
:105B300003E113E00FC0E114F10409F06052D30156
:105B4000ED91FC910190F081E02DC10109950F5F6D
:105B50001F4F05C0EF2CFF24B0E1EB22FF24F8011A
:105B60006491662341F748C1F7FE13C0BC0CFE8563
:105B7000F4FF04C08A81813309F4BA941B141CF029
:105B8000BB24B3942DC048E04B1550F538E0B32E3C
:105B900027C0F6FC25C0892D90E08C159D054CF0A2
:105BA0005CEFC5165FEFD50624F080E8F82A01C047
:105BB0009A94992049F0E2E0F0E0EC0FFD1FE90D26
:105BC000F11D80818033A1F3F7FE0AC0B92CB39494
:105BD000892D90E0C816D90614F0992401C09C18AC
:105BE000F7FC03C025E030E009C01C141D041CF0C4
:105BF00021E030E003C096012F5F3F4F112311F0E9
:105C00002F5F3F4F992029F0892D90E00196280FB2
:105C1000391F882D90E02817390714F0882401C017
:105C2000821A4F2C5524C20189709070892B59F02B
:105C30000CC0D301ED91FC910190F081E02DC101E8
:105C400060E209958A948820A1F7112349F0D301D5
:105C5000ED91FC910190F081E02DC101612F09953A
:105C600043FE0BC00CC0D301ED91FC910190F0817B
:105C7000E02DC10160E309958A948820A1F7F7FE21
:105C800051C08601D7FE02C000E010E07601089402
:105C9000E11CF11CE01AF10AE1E0F0E0EC0FFD1F5D
:105CA000EE0EFF1E26014B185108892D90E0AA2404
:105CB000BB24A81AB90AFFEF0F3F1F0749F4D3010D
:105CC000ED91FC910190F081E02DC1016EE209950A
:105CD000C016D10634F0401651061CF4F70160815D
:105CE00001C060E3015010400894E11CF11C0A154A
:105CF0001B054CF0D301ED91FC910190F081E02D5A
:105D0000C1010995D8CF0C151D0541F48A81863350
:105D100020F4853319F4BE85B4FF61E3D301ED911E
:105D2000FC9165C06A81613309F00F7ED301ED916A
:105D3000FC910190F081E02DC10109959920E1F0DD
:105D4000D301ED91FC910190F081E02DC1016EE253
:105D5000099512E0E1E0F0E0EC0FFD1FE10FF11D0D
:105D600060811F5FD301ED91FC910190F081E02DE6
:105D7000C10109959A9471F7D301ED91FC910190BD
:105D8000F081E02D44FC02C065E601C065E4C1017C
:105D90000995D7FC05C0C114D10441F404FF06C025
:105DA000D094C194D108D3946DE201C06BE2D301C9
:105DB000ED91FC910190F081E02DC101099560E326
:105DC00005C06F5FE6EFFFEFCE0EDF1EFAE0CF16E5
:105DD000D104BCF7D301ED91FC910190F081E02D4D
:105DE000C1010995D301ED91FC916C2D605D01908D
:105DF000F081E02DC1010995CC84DD8478C1933612
:105E000031F0933799F0933509F061C023C0F60162
:105E1000808189835E010894A11CB11C42E050E09E
:105E2000C40ED51E21E0E22EF12C12C0D601AD9099
:105E3000BC9016FD03C06FEF7FEF02C0692D70E0CC
:105E4000E2E0F0E0CE0EDF1EC5010E9428047C01D6
:105E50001F7713C0D601AD90BC9016FD03C06FEF45
:105E60007FEF02C0692D70E0E2E0F0E0CE0EDF1EB1
:105E7000C5010E941D047C01106813FF0BC023C0E4
:105E8000D301ED91FC910190F081E02DC10160E220
:105E900009958A94882D90E0E816F90688F313C0D6
:105EA000F50117FD659117FF61915F01D301ED9138
:105EB000FC910190F081E02DC101099581108A9437
:105EC0000894E108F108E114F10451F710C1943687
:105ED00011F0993699F517FF0AC0F601208131813A
:105EE0004281538184E090E0C80ED91E0CC0D601D7
:105EF0008D919C919C01442737FD4095542FE2E001
:105F0000F0E0CE0EDF1E9FE6F92EF12257FF09C00A
:105F100050954095309521953F4F4F4F5F4FF0E89A
:105F2000FF2ACA01B901AE014F5F5F4F2AE030E09E
:105F30000E94E501E82E4B89E41A41C0953721F40F
:105F40001F7E2AE030E01CC0197F9F3661F0903739
:105F500020F4983509F0CEC00FC0903739F098374B
:105F600009F0C8C004C028E030E00AC0106114FD88
:105F7000146020E130E004C014FD166020E132E03E
:105F800017FF08C0D6016D917D918D919C91E4E041
:105F9000F0E008C0D6018D919C91BC0180E090E0BA
:105FA000E2E0F0E0CE0EDF1EAE014F5F5F4F0E94D9
:105FB000E501E82EFB89EF1A8FE7F82EF122F6FEB5
:105FC0000BC04EEFF422E91438F4F4FE07C0F2FCE3
:105FD00005C05FEEF52202C01E2D01C0192DF4FE92
:105FE0000DC0FE01EE0DF11D8081803319F489EEA4
:105FF000F82208C01F5FF2FE05C003C08F2D86780F
:1060000009F01F5F0F2DF3FC18C0F0FE13C0181528
:1060100010F09E2C0FC09E2C980C911A182D0AC0BF
:10602000D301ED91FC910190F081E02DC10160E27E
:1060300009951F5F1815A0F304C0181510F4811AF4
:1060400001C0882404FF17C0D301ED91FC91019099
:10605000F081E02DC10160E3099502FF29C0D30161
:10606000ED91FC910190F081E02D01FD02C068E707
:1060700012C068E510C0802F8678D1F001FF02C001
:106080006BE201C060E2F7FC6DE2D301ED91FC919F
:106090000190F081E02DC10109950AC0D301ED9175
:1060A000FC910190F081E02DC10160E309959A9483
:1060B000E914A0F3EA94D301ED91FC91A1E0B0E0E2
:1060C000AC0FBD1FAE0DB11D0190F081E02DC101DF
:1060D0006C910995EE2071F70AC0D301ED91FC9106
:1060E0000190F081E02DC10160E209958A94882039
:1060F000A1F71DCC64960FB6F894DEBF0FBECDBFDE
:10610000CF91DF911F910F91FF90EF90DF90CF9093
:10611000BF90AF909F908F907F906F905F904F90C7
:106120003F902F900895F999FECF72BD61BDF89A06
:1061300080B50895F999FECF1FBA72BD61BD40BD0B
:106140000FB6F894FA9AF99A0FBE08950F93FC01CE
:106150006115710511F480E011C0218332834383FE
:106160005483728761870170000F000F000F8081D8
:10617000877F802B82608B7F808381E00F910895E1
:10618000CF93DF93EC010E947B319B01AC018D81A9
:106190009E81AF81B885281739074A075B0728F425
:1061A000888184FD02C060E00DC089819A81AB8145
:1061B000BC81820F931FA41FB51F8D839E83AF8365
:1061C000B88761E0222757FD2395332744275527B9
:1061D000922F91709295907F88818F7E892B8883F2
:1061E000862FDF91CF910895CF93DF93EC018881C3
:1061F00082FF0FC0CE010E94C030882351F0E98594
:10620000FA85309709F00995888183FF02C08B7F5A
:106210008883DF91CF910895CF93DF93EC01898537
:106220009A85892BE1F089819A81AB81BC810097A5
:10623000A105B105A1F00E947B3129813A814B81F2
:106240005C81260F371F481F591F2D833E834F83C4
:106250005887888184608F7E888381E001C080E0D8
:10626000DF91CF9108951F920F920FB60F921124D4
:106270002F933F938F939F93AF93BF938091A606E5
:106280009091A706A091A806B091A9063091AA0600
:106290000196A11DB11D232F2D5F2D3720F02D5705
:1062A0000196A11DB11D2093AA068093A606909386
:1062B000A706A093A806B093A9068091A206909184
:1062C000A306A091A406B091A5060196A11DB11D3B
:1062D0008093A2069093A306A093A406B093A5066C
:1062E000BF91AF919F918F913F912F910F900FBED2
:1062F0000F901F9018958FB7F8942091A6063091B3
:10630000A7064091A8065091A9068FBFB901CA01FE
:1063100008959B01AC017FB7F8948091A2069091FB
:10632000A306A091A406B091A50666B5A89B05C0DA
:106330006F3F19F00196A11DB11D7FBFBA2FA92F84
:10634000982F8827860F911DA11DB11D62E0880F2F
:10635000991FAA1FBB1F6A95D1F7BC012DC0FFB7BB
:10636000F8948091A2069091A306A091A406B09102
:10637000A506E6B5A89B05C0EF3F19F00196A11D43
:10638000B11DFFBFBA2FA92F982F88278E0F911DFF
:10639000A11DB11DE2E0880F991FAA1FBB1FEA953E
:1063A000D1F7861B970B885E9340C8F2215030408E
:1063B0004040504068517C4F211531054105510541
:1063C00071F60895019739F0880F991F880F991F6A
:1063D00002970197F1F70895789484B5826084BD9F
:1063E00084B5816084BD85B5826085BD85B58160D9
:1063F00085BDEEE6F0E0808181608083E1E8F0E039
:106400001082808182608083808181608083E0E867
:10641000F0E0808181608083E1EBF0E08081846046
:106420008083E0EBF0E0808181608083EAE7F0E048
:1064300080818460808380818260808380818160AC
:1064400080838081806880831092C10008951F92AC
:106450000F920FB60F9211242F933F934F935F9398
:106460006F937F938F939F93AF93BF93EF93FF931C
:106470008091AB069091AC06892B29F0E091AB0698
:10648000F091AC060995FF91EF91BF91AF919F916B
:106490008F917F916F915F914F913F912F910F90CD
:1064A0000FBE0F901F9018951F920F920FB60F926C
:1064B00011242F933F934F935F936F937F938F9309
:1064C0009F93AF93BF93EF93FF938091AD0690910D
:1064D000AE06892B29F0E091AD06F091AE06099544
:1064E000FF91EF91BF91AF919F918F917F916F91AC
:1064F0005F914F913F912F910F900FBE0F901F9082
:106500001895CF93DF93482F50E0CA01875B9C4FCB
:10651000FC0134914B5C5C4FFA018491882369F152
:1065200090E0880F991FFC01E95EFC4FA591B491A2
:10653000FC01EF5DFC4FC591D491662351F42FB758
:10654000F8948C91932F909589238C93888189233B
:106550000BC0623061F42FB7F8948C91932F909513
:1065600089238C938881832B88832FBF06C09FB794
:10657000F8948C91832B8C939FBFDF91CF910895DA
:10658000482F50E0CA01835A9C4FFC012491CA0154
:10659000875B9C4FFC0194914B5C5C4FFA013491FA
:1065A000332309F440C0222351F1233071F0243009
:1065B00028F42130A1F0223011F514C02630B1F0BA
:1065C0002730C1F02430D9F404C0809180008F7747
:1065D00003C0809180008F7D8093800010C084B5BF
:1065E0008F7702C084B58F7D84BD09C08091B000D3
:1065F0008F7703C08091B0008F7D8093B000E32F30
:10660000F0E0EE0FFF1FEF5DFC4FA591B4912FB7A7
:10661000F894662321F48C919095892302C08C9183
:10662000892B8C932FBF08958093B0020895982FE3
:106630008E3008F09E5097708091B0028295880F3E
:10664000880F807C892B80937C0080917A00806405
:1066500080937A0080917A0086FDFCCF20917800AB
:1066600040917900942F80E030E0282B392BC9012C
:106670000895CF92DF92EF92FF920F931F93CF93E3
:10668000DF937C016B018A01C0E0D0E00FC0D6012E
:106690006D916D01D701ED91FC910190F081E02D9C
:1066A000C7010995C80FD91F0150104001151105E8
:1066B00071F7CE01DF91CF911F910F91FF90EF9075
:1066C000DF90CF900895CF93DF930E94EC310E942A
:1066D0009B27C0E0D0E00E94C2292097E1F30E94EE
:1066E0000000F9CF5058BB27AA270ED041C201D2D3
:1066F00030F006D220F031F49F3F11F41EF4C0C1F7
:106700000EF4E095E7FBB6C1E92F54D280F3BA1737
:10671000620773078407950718F071F49EF56CC241
:106720000EF4E0950B2EBA2FA02D0B01B9019001AC
:106730000C01CA01A0011124FF27591B99F0593FF0
:1067400050F4503E68F11A16F040A22F232F342F38
:106750004427585FF3CF469537952795A795F04086
:106760005395C9F77EF41F16BA0B620B730B840B9B
:10677000BAF09150A1F0FF0FBB1F661F771F881F53
:10678000C2F70EC0BA0F621F731F841F48F48795AB
:1067900077956795B795F7959E3F08F0B3CF93959A
:1067A000880F08F09927EE0F979587950895A1D146
:1067B00058F080E891E009F49EEFA2D128F040E87B
:1067C00051E059F45EEF09C05BC116C2E92FE078D1
:1067D000F1D168F3092E052AC1F3261737074807B8
:1067E000590738F00E2E07F8E02569F0E025E0643F
:1067F0000AC0EF6307F8009407FADB01B9019D01B5
:10680000DC01CA01AD01EF934AD0B2D10AD05F9149
:10681000552331F02BED3FE049E450FD49EC63CFC7
:106820000895DF93DD27B92FBF7740E85FE31616A1
:10683000170648075B0710F4D92FE9D19F938F9370
:106840007F936F93BCD2E8E6F0E01DD191D12F91F8
:106850003F914F915F91EED1DD2349F09058A2EA2C
:106860002AED3FE049EC5FE3D0785D274DDFDF9113
:106870007FC1DCD008F481E008954AD1E39589C155
:106880000CD076C13DD140F034D130F021F45F3FDF
:1068900019F0F0C05111B1C1F3C08CD198F3992314
:1068A000C9F35523B1F3951B550BBB27AA276217D4
:1068B0007307840738F09F5F5F4F220F331F441F19
:1068C000AA1FA9F333D00E2E3AF0E0E830D0915051
:1068D0005040E695001CCAF729D0FE2F27D0660F3E
:1068E000771F881FBB1F261737074807AB07B0E87D
:1068F00009F0BB0B802DBF01FF2793585F4F2AF093
:106900009E3F510568F0B6C078C15F3FECF3983EFA
:10691000DCF3869577956795B795F7959F5FC9F7EF
:10692000880F911D9695879597F90895E1E0660F78
:10693000771F881FBB1F621773078407BA0720F0F1
:10694000621B730B840BBA0BEE1F88F7E09508955A
:1069500004D06894B11151C1089534D188F09F5783
:1069600090F0B92F9927B751A0F0D1F0660F771F9B
:10697000881F991F1AF0BA95C9F712C0B13081F07B
:106980003BD1B1E0089538C1672F782F8827B85FD1
:1069900039F0B93FCCF3869577956795B395D9F7DC
:1069A0003EF490958095709561957F4F8F4F9F4FE6
:1069B0000895E89409C097FB3EF4909580957095F2
:1069C00061957F4F8F4F9F4F9923A9F0F92F96E93B
:1069D000BB279395F695879577956795B795F111B0
:1069E000F8CFFAF4BB0F11F460FF1BC06F5F7F4F4D
:1069F0008F4F9F4F16C0882311F096E911C077235F
:106A000021F09EE8872F762F05C0662371F096E867
:106A1000862F70E060E02AF09A95660F771F881F36
:106A2000DAF7880F9695879597F90895990F0008DA
:106A3000550FAA0BE0E8FEEF16161706E807F90750
:106A4000C0F012161306E407F50798F0621B730BEB
:106A5000840B950B39F40A2661F0232B242B252B6C
:106A600021F408950A2609F4A140A6958FEF811D0F
:106A7000811D089597F99F6780E870E060E00895B0
:106A80009FEF80EC0895DF93CF931F930F93FF92B6
:106A9000EF92DF927B018C01689405C0DA2EEF0142
:106AA000C9D0FE01E894A591259135914591559164
:106AB000AEF3EF0129DEFE019701A801DA9479F720
:106AC000DF90EF90FF900F911F91CF91DF9108958C
:106AD0009F938F937F936F93FF93EF939B01AC01F1
:106AE0009DD0EF91FF91CFDF2F913F914F915F911B
:106AF00095C000240A94161617061806090608956C
:106B000000240A9412161306140605060895B8CF39
:106B100059D0E8F3E894EFEFBB273FE048EC5FE79C
:106B20006B3D73078407950708F1FF279F57B25AFB
:106B30006A4D7F40894CF04032F4BE556542704F3B
:106B40008643FF4F0894EE1F915030F0BB0F661F35
:106B5000771F881FFF1FEBCF9EE7882332F0BB0F04
:106B6000661F771F881F9A95C1F79395E09565C1B9
:106B7000092E0394000C11F4882352F0BB0F40F44B
:106B8000BF2B11F460FF04C06F5F7F4F8F4F9F4F8B
:106B90000895EF93E0FF06C0A2EA2AED3FE049EC3A
:106BA0005FEBB2DDE5DF0F90039401FC9058E5E95F
:106BB000F0E08ECF57FD9058440F551F59F05F3FBE
:106BC00071F04795880F97FB991F61F09F3F79F00F
:106BD00087950895121613061406551FF2CF469591
:106BE000F1DF08C0161617061806991FF1CF869513
:106BF0007105610508940895E894BB2766277727F7
:106C0000CB0197F9089512DF08F48FEF08959B01E7
:106C1000AC0160E070E080E89FE332CE0BD0A8CFFB
:106C200068DF28F06DDF18F0952309F023CF28CF17
:106C30001124E3CFBFDFA0F3959FD1F3950F50E070
:106C4000551F629FF001729FBB27F00DB11D639F1E
:106C5000AA27F00DB11DAA1F649F6627B00DA11DC4
:106C6000661F829F2227B00DA11D621F739FB00D6A
:106C7000A11D621F839FA00D611D221F749F3327DA
:106C8000A00D611D231F849F600D211D822F762F73
:106C90006A2F11249F5750408AF0E1F088234AF070
:106CA000EE0FFF1FBB1F661F771F881F91505040BC
:106CB000A9F79E3F510570F0DDCE9FCF5F3FECF30B
:106CC000983EDCF3869577956795B795F795E795A8
:106CD0009F5FC1F7FE2B880F911D9695879597F9B9
:106CE000089570DFE0F09E37D8F09639B8F49E38FA
:106CF00048F4672F782F8827985FF9CF8695779586
:106D0000679593959539D0F3B62FB1706B0F711DC0
:106D1000811D20F4879577956795939573C08DC0F5
:106D20006CCF11F40EF4ACCE88C04CDFD0F39923B5
:106D3000D9F3CEF39F57550B87FF8FD05695979574
:106D4000B0E020F4660F771F881FBB1F1F930F93BF
:106D500000249001A0018001F001A0E80E0F1F1F88
:106D60000A1E511D601B710B8009B50B48F4600FA2
:106D7000711F801DB51F0E1B1F0B0A0A510907C08A
:106D80002E0F3F1F4A1F0E0F1F1F0A1E511D660F99
:106D9000771F881FBB1FA695F795E795F8F606178E
:106DA000170708065B07211D311D411D0F911F911B
:106DB000B901842F9158880F9695879508959B0166
:106DC000AC012CCFDF93D92FA3DEE695D7952AED22
:106DD0003FE049E45FE3B33A62077307840795072E
:106DE000D7952AF0A2EA49EC90688EDCC1DEE3EB8D
:106DF000F0E06EDEDD0F0BF00ADFDD0F0BF49058D4
:106E0000DF910895882371F4772321F09850872B20
:106E1000762F07C0662311F499270DC09051862B59
:106E200070E060E02AF09A95660F771F881FDAF706
:106E3000880F9695879597F908959F3F49F091504F
:106E400028F4869577956795B7959F5F80389F4F13
:106E5000880F9695879597F9089591505040660F41
:106E6000771F881FD2F70895AA1BBB1B51E107C0EB
:106E7000AA1FBB1FA617B70710F0A61BB70B881FCA
:106E8000991F5A95A9F780959095BC01CD01089559
:106E900097FB092E07260AD077FD04D0E5DF06D040
:106EA00000201AF4709561957F4F0895F6F790953C
:106EB00081959F4F0895A1E21A2EAA1BBB1BFD01CD
:106EC0000DC0AA1FBB1FEE1FFF1FA217B307E407C9
:106ED000F50720F0A21BB30BE40BF50B661F771F21
:106EE000881F991F1A9469F7609570958095909501
:106EF0009B01AC01BD01CF01089597FB092E05262A
:106F00000ED057FD04D0D7DF0AD0001C38F45095BE
:106F10004095309521953F4F4F4F5F4F0895F6F7BD
:106F200090958095709561957F4F8F4F9F4F0895F5
:106F3000EE0FFF1F0590F491E02D0994F894FFCF18
:106F400025630025632563002563253269256325B4
:106F50003032697C2563253269256325303269002A
:106F600025352E3066256300256325312E356625AF
:106F700063002563253569256300256325352E3299
:106F8000662563006D616E007374310073743200A6
:106F90007374330073743400737435007374360083
:106FA00070682000636C200076722000686C2000FE
:106FB00061702000727462006C616E00707020005D
:106FC000706F6900616320000061742000256325F3
:106FD0007300256325332E30692563002534692528
:106FE00063256300256325336925630025737C25AC
:106FF00063257325630020C0C0C0C0C0C7C0C0C027
:10700000C0C0200025342E3066256300256325335B
:107010002E3066256300256325352E3066256300F6
:1070200025632531312E36667C25632531312E3698
:10703000660025632532690025332E3166256300FD
:10704000202020202020202020202020002020641C
:10705000697361726D6564202000206E6F20746515
:107060006C20636F6D2000206E6F20677073206648
:1070700069782000202062617474206C6F77202072
:107080000062617474207761726E696E670062617C
:107090007474637269746963616C002062617474F2
:1070A000206572726F7220006C696E6B2071756161
:1070B0006C697479006D6167207761726E696E67C3
:1070C000006D616720637269746963616C00206D93
:1070D000616720206572726F7220002573002000A6
:1070E000B3060000E803E803E803E8039DFF01643A
:1070F00001000000007B05393379047C047F0482A1
:1071000004CE2900070E091C1B1215383F36312406
:10711000232A2D70777E796C6B6265484F46415407
:10712000535A5DE0E7EEE9FCFBF2F5D8DFD6D1C4B7
:10713000C3CACD90979E998C8B8285A8AFA6A1B427
:10714000B3BABDC7C0C9CEDBDCD5D2FFF8F1F6E3D8
:10715000E4EDEAB7B0B9BEABACA5A28F8881869347
:10716000949D9A2720292E3B3C35321F1811160377
:10717000040D0A5750595E4B4C45426F6861667367
:10718000747D7A898E878095929B9CB1B6BFB8AD8D
:10719000AAA3A4F9FEF7F0E5E2EBECC1C6CFC8DD87
:1071A000DAD3D4696E676075727B7C51565F584D37
:1071B0004A4344191E171005020B0C21262F283DA7
:1071C0003A33344E49404752555C5B7671787F6A5A
:1071D0006D64633E39303722252C2B0601080F1AC7
:1071E0001D1413AEA9A0A7B2B5BCBB9691989F8AF7
:1071F0008D8483DED9D0D7C2C5CCCBE6E1E8EFFAE7
:10720000FDF4F3C2C0C0C1C0C0C1C0C0C4C0C0C1D1
:10721000C0C0C1C0C0C3C0C0C1C0C0C1C0C0C5C063
:10722000C0C1C0C0C1C0C000000000E42A3933554D
:107230002A852AB52AD22A6B2AF329392BA92B00B1
:00000001FF
